:106CA6000000050200000301FA0400FA0500030AC9
:106CB6000A5A0B001E0C00FA0D00030E00040F0109
:106CC60064100096120132130AFA14010217010A1F
:106CD6001801FA1905321A010A1B01FA1C05321F9E
:106CE600FFFF20FFFF23011E2400642A00FA2B0069
:106CF600FA2C50782D003D2E004630006432507834
:106D06003300003432FA35016436016437015038F5
:106D16000A643C00643E003C3F000140FFFF411412
:106D260050420A5A430AC84405324500B44600FA9E
:106D36004C00FA500808510596520A32530B465435
:106D46000A96570546590A465A32FA5B010A5C0A00
:106D5600325E000A5F00FE64021C67FFFF6A0A3C9F
:106D66006B00006C32967300017400017801327971
:106D760001327E006481006484FFFF8A00019D0A5F
:106D8600969E00019FFFFFA0013CA2000AA3FFFF01
:106D9600A4FFFFA5FFFFA6FFFFA7FFFFA8FFFFA910
:106DA600FFFF01013C1500022F003C470178480215
:106DB600035601024EFFFF58000261FFFF66000204
:106DC6008500AF8600018700FA89010A990008A1AB
:106DD60000FAFAFAFA01013C1500022F1E3C47019F
:106DE600784802035601024EFFFF58000261FFFF7A
:106DF6006600028500AF8600018700FA89010A99BC
:106E06000000A10000FAFAFA01013C1500002F1E4D
:106E16003C47013C4802025601014EFFFF58000064
:106E260061FFFF66000085FFFF86FFFF87FFFF8982
:106E36000102990000A10000FAFAFA0065006F004D
:106E4600790083008D009700A100AC00B600C00059
:106E5600CA00D400DE00E800F200580060006800B6
:106E6600700078008000880090009800A000A800BC
:106E7600B000B800C100C800D000D800DF00E600AE
:106E8600EE00F600410047004D00530059005F0038
:106E960065006C00710077007D00830089008F001B
:106EA60095009B00A200A700AC00B200B900C0008C
:0F6EB600C500CA00D200D500DD00E100E700EF03
:10009E0090089AE0900126F090089BE0900095F071
:1000AE0090089CE09000B5F090089DE09000DEF086
:1000BE0090089EE090008AF090089FE09000D0F0AB
:1000CE009008A0E09000EEF09008A1E09000C2F041
:1000DE009008A2E09000E0F09008A3E0900110F0EC
:1000EE009008A4E0900174F09008A5E0900175F0DE
:1000FE009008A6E0900176F0900174E0700C9001EB
:10010E0075E07006900176E060028004C2248002E1
:10011E00D224743690015FF07430900160F0742D2B
:10012E00900161F07432900162F07420900163F0DE
:10013E007438900164F07443900165F07479900105
:10014E0066F0746C900167F07420900168F0742072
:10015E00900169F0742090016AF0742090016BF0A8
:10016E00742090016CF0742090016DF02290089232
:10017E00E0FEA3E0FF7402D39F74019E400C906CCE
:10018E00A6120048E493F599804C900061E0D39458
:10019E00054014900892E0FEA3E0FF906CA61200BA
:1001AE0048E493F599802F900061E0D394044014B5
:1001BE00900892E0FEA3E0FF906CD9120048E49301
:1001CE00F5998012900892E0FEA3E0FF906D0C125C
:1001DE000048E493F599900892126FE5900892E02A
:1001EE00FEA3E0FFEFB43507EEB40103754D002218
:1001FE0085F97385FA747E017F00E574126FD7E579
:10020E00732FFF50010E8E5A8F5B90001DE0FCA3E2
:10021E00E0FDEF2DFDEE3CFC8C5C8D5D2275A71094
:10022E0085F97385FA747E017F00E574126FD7E548
:10023E00732FFF50010E8E5A8F5B90001DE0FCA3B2
:10024E00E0FDEF2DFDEE3CFC8C5C8D5D22E55DF559
:10025E00FBE55CF5FCD29322E55DF5E9E55CF5EA9C
:10026E00D29422E55DF5EBE55CF5ECD29122E55DED
:10027E00F5EDE55CF5EED29222E55DF5FBE55CF57C
:10028E00FCD28722E55DF5E9E55CF5EAD29022E540
:10029E005DF5EBE55CF5ECE5B54410F5B522E55DF5
:1002AE00F5EDE55CF5EEE5B54420F5B522AE5AAFB9
:1002BE005B74068E048F05FF126FC78C5C8D5DAE6E
:1002CE005AAF5B74068E048F05FF126FF28C5A8D37
:1002DE005BE55B455A60137406C3955BFFE4955A64
:1002EE00FE8E5A8F5B785C12702AE573A85CB8009C
:1002FE0015D3955D4010E573C3955DFFE4955CFEE7
:10030E008E5C8F5D8010E573243CC3955DFFE49594
:10031E005CFE8E5C8F5DAE5CAF5D743B6F4E6006B7
:10032E00743C6F4E701AAE5CAF5D743B6F4E7005D1
:10033E007573018003757302755D3A755C008003F9
:10034E007573002290009CE0B40104C2068002D2B4
:10035E000690009DE0B40104C2078002D20790000F
:10036E00DAE075F0E1A4FFAEF0740A8E048F05FF9B
:10037E00126FC790088AECF0A3EDF074078C068D0F
:10038E0007126FD774038E048F05FF126FC790008C
:10039E0019ECF0A3EDF07E017F00900098E0126F53
:1003AE00D79000DBE08E048F05FF126FC7740AFF33
:1003BE00126FC78D609000E4E075F0E1A4FFAEF01F
:1003CE00740A8E048F05FF126FC790088EECF0A38F
:1003DE00EDF09000E6E060139000E6E0F5F07416A4
:1003EE0084FF7E00EF9008B6F0800674649008B625
:1003FE00F09000DCE0900078F0900128E090008210
:10040E00F090012AE0FE9000D8E08E0088F0A4FF64
:10041E00AEF0EF9008BEF0900126E090089AF090B2
:10042E0000B5E090089CF09000DEE090089DF09002
:10043E00008AE090089EF0900110E09008A3F090E2
:10044E000174E09008A4F0900175E09008A5F0907A
:10045E000176E09008A6F0A224B34016900174E055
:10046E00700C900175E07006900176E060028002DB
:10047E00C224900174E0B4300F900175E0B44708C7
:10048E00900176E0643B60028004D2258002C22592
:10049E0074E3900077F09000C5E0B40B0874E3901D
:1004AE000077F0805A9000C5E0B419129000DBE09E
:1004BE00906E2C12008CE493900077F080419000A7
:1004CE00C5E0B41E129000DBE0906E4A12008CE480
:1004DE0093900077F080289000C5E0B42812900029
:1004EE00DBE0906E7412008CE493900077F0800F36
:1004FE009000C5E0B446089000BCE0900077F09004
:10050E00007BE0FE9000C2E0B5064B90007DE0FE61
:10051E009000E0E0B5063F90007CE0FE9000EEE03B
:10052E00B5063390007FE0FE900095E0B50627906B
:10053E00007EE0FE9000D0E0B5061B900080E0FE4D
:10054E009000FBE0B5060F900081E0FE9000FCE00D
:10055E006E7003020773900061E0C3940550087437
:10056E0002900111F0801C9000D0E06403600690B0
:10057E0000EEE060087406900111F08006740A9097
:10058E000111F09000D0E0B403089000EEE0640298
:10059E006002800674009000EEF0900095E0B401C9
:1005AE00067400900095F0900095E0B40206740079
:1005BE009000E0F0900095E0B4030674009000ED1A
:1005CE00F09000C2E0601474299000A9F0740090BD
:1005DE0006CEF074009006CFF0800C74009000A947
:1005EE00F074299006CEF09000C2E0B40214742A82
:1005FE009000AAF074009006D2F074009006D3F02A
:10060E00800C74009000AAF0742A9006D2F090002C
:10061E00FBE060147419900115F074009006D6F08A
:10062E0074009006D7F0800C7400900115F07419C8
:10063E009006D6F09000FCE06014741A900116F04B
:10064E0074009006DAF074009006DBF0800C7400F3
:10065E00900116F0741A9006DAF09000E0E0D39450
:10066E00014014741B900113F074009006DEF074B8
:10067E00009006DFF0800C7400900113F0741B9054
:10068E0006DEF09000EEE0B40114741C900114F03C
:10069E0074009006E2F074009006E3F0800C740093
:1006AE00900114F0741C9006E2F09000D0E0B402B9
:1006BE00069000EEE06002801A74059006E6F07473
:1006CE00069006EAF074079006EEF074089006F2B3
:1006DE00F0803074009006E6F074009006E7F07437
:1006EE00009006EAF074009006EBF074009006EEAF
:1006FE00F074009006EFF074009006F2F074009023
:10070E0006F3F0D2239000C2E090007BF09000EE52
:10071E00E090007CF09000E0E090007DF09000D042
:10072E00E090007EF0900095E090007FF09000FB4E
:10073E00E0900080F09000FCE0900081F090009539
:10074E00E090089BF09000D0E090089FF09000EEB3
:10075E00E09008A0F09000C2E09008A1F09000E0B8
:10076E00E09008A2F09000F8E0B401179000297410
:10077E000FF0A374FFF090002BE4F0A3F07402903E
:10078E0000F8F09000F8E0B4034190002BE0FEA3D7
:10079E00E0FF900029E0FCA3E0FD1270227410121D
:1007AE006FD77408120039EF900074F0EF70067472
:1007BE00FF900074F074009000F8F090002AE09022
:1007CE000075F0900029E0900076F0900089E0909E
:1007DE000086F0900088E0900085F09000B7E0C3AE
:1007EE00941E50569000B7E0F404241E900087F03B
:1007FE00900087E075F00684FF7E008F739000876F
:10080E00E075F00684ADF07C008D74900085E0D329
:10081E009574400D900085E0C39574900085F0802E
:10082E000F900085E02406C39574900085F0057343
:10083E00900086E02573900086F0900086E0900090
:10084E004DF090004DE0D3943C400B90004DE0C332
:10085E00943C90004DF090004DE0240F90004EF02F
:10086E0090004DE0241E90004FF090004DE0242D9E
:10087E00900050F090004EE0D3943C400B90004E10
:10088E00E0C3943C90004EF090004FE0D3943C4077
:10089E000B90004FE0C3943C90004FF0900050E05E
:1008AE00D3943C400B900050E0C3943C900050F029
:1008BE00900055E4F090004DE0643B600790004DD1
:1008CE00E0B43C2090004DE0B43B0674029000551D
:1008DE00F090004DE0B43C069000557401F090008D
:1008EE004D7401F0900056E4F090004EE0643B60D1
:1008FE000790004EE0B43C2090004EE0B43B0674EE
:10090E0002900056F090004EE0B43C0690005674F3
:10091E0001F090004E7401F0900057E4F090004FFB
:10092E00E0643B600790004FE0B43C2090004FE045
:10093E00B43B067402900057F090004FE0B43C06B2
:10094E009000577401F090004F7401F0900058E43D
:10095E00F0900050E0643B6007900050E0B43C2003
:10096E00900050E0B43B067402900058F090005096
:10097E00E0B43C069000587401F09000507401F001
:10098E00900089E0FE9000ECE02E90005AF090006E
:10099E005AE0641E600790005AE0B43C0690005A7C
:1009AE00E004F090005AE0641D600790005AE0B435
:1009BE003B0690005AE014F090005AE0D3943C406D
:1009CE000B90005AE0C3943C90005AF090005AE00D
:1009DE00D3941E400D90005AE0C3941E90005BF01D
:1009EE00800A90005AE0241E90005BF075511E9014
:1009FE0000CFE0900051F0900051E075F00F84AF01
:100A0E00F07E00EF4E7006900051E004F090005121
:100A1E00E00475F00F84AFF07E00EF4E700690008C
:100A2E0051E014F0900051E0B47906900051740139
:100A3E00F0900051E0D3943C400F900051E0C394ED
:100A4E003C900051F0D21E8002C21E900051E02454
:100A5E000F900052F0900051E0241E900053F09041
:100A6E000051E0242D900054F0900052E0D3943CBD
:100A7E00400B900052E0C3943C900052F090005313
:100A8E00E0D3943C400B900053E0C3943C90005351
:100A9E00F0900054E0D3943C400B900054E0C3948B
:100AAE003C900054F022C293C294C291C292C2876B
:100ABE00C290E5B554EFF5B5E5B554DFF5B5C29680
:100ACE00C295C2A0C297C2A2C2A1E5B554BFF5B5E8
:100ADE00E5B5547FF5B5E5B554FBF5B5C208755EC1
:100AEE00469000D2E07005756D028003756D03753A
:100AFE00550075540090001074FFF0A374DCF0C222
:100B0E000FC211C213C21574C890003DF074C89084
:100B1E000041F074C8900045F074C8900049F0751B
:100B2E005300755200C203754600E56FB409037594
:100B3E006F0075630090001FE4F0A3F0757010C293
:100B4E000BC20CC20DC20EC2027557007556009034
:100B5E000012E4F0A3F0900014E4F0A3F0C22975A3
:100B6E005900755800900094E075F032A4FFAEF075
:100B7E00900027EEF0A3EFF0900083E4F090008455
:100B8E00E4F0C226D21BC21AD21CC21DC21EC21F44
:100B9E0022755B00755A00AE5AAF5B7402C39F7428
:100BAE00019E5003020C5D906CA6120048E49390D7
:100BBE0000881270080FBF00010EE0FC906CA612A8
:100BCE000048ECFEE493FFEEC39F5026AE5AAF5B97
:100BDE000FBF00010E906CA6120048AE5AAF5BE438
:100BEE0093FC906CA6120048E49390008812700853
:100BFE00ECF0AE5AAF5B906CA6120048E4939000F6
:100C0E0088127008E0FC906CA8120048ECFCE4938B
:100C1E00FDECD39D4019906CA8120048E493FC9013
:100C2E006CA6120048E493900088127008ECF0AEA7
:100C3E005AAF5B74022FFF50010E8E5A8F5B785B9A
:100C4E00740126F6500418E436F64003020BA52272
:100C5E00755B00755A00AE5AAF5B7433BE00039FCE
:100C6E005003020D2B906DA8120048E4939000885B
:100C7E001270080FBF00010EE0FC906DA812004824
:100C8E00ECFEE493FFEEC39F5026AE5AAF5B0FBF50
:100C9E0000010E906DA8120048AE5AAF5BE493FCB3
:100CAE00906DA8120048E493900088127008ECF042
:100CBE00AE5AAF5B906DA8120048E4939000881274
:100CCE007008E0FC906DAA120048ECFCE493FDEC79
:100CDE00D39D4019906DAA120048E493FC906DA824
:100CEE00120048E493900088127008ECF0AE5AAFF0
:100CFE005B742D6F4E7006755B33755A00AE5AAF2E
:100D0E005B74022FFF50010E8E5A8F5B785B74015D
:100D1E0026F6500418E436F64003020C6422755B86
:100D2E0000755A00AE5AAF5B7433BE00039F50037A
:100D3E00020DF9906DDB120048E49390008812705A
:100D4E00080FBF00010EE0FC906DDB120048ECFEB8
:100D5E00E493FFEEC39F5026AE5AAF5B0FBF000168
:100D6E000E906DDB120048AE5AAF5BE493FC906DB3
:100D7E00DB120048E493900088127008ECF0AE5A33
:100D8E00AF5B906DDB120048E49390008812700800
:100D9E00E0FC906DDD120048ECFCE493FDECD39D7D
:100DAE004019906DDD120048E493FC906DDB12004B
:100DBE0048E493900088127008ECF0AE5AAF5B7462
:100DCE002D6F4E7006755B33755A00AE5AAF5B745D
:100DDE00022FFF50010E8E5A8F5B785B740126F640
:100DEE00500418E436F64003020D3222755B00758E
:100DFE005A00AE5AAF5B7433BE00039F5003020E0F
:100E0E00C7906E0E120048E4939000881270080F7F
:100E1E00BF00010EE0FC906E0E120048ECFEE49353
:100E2E00FFEEC39F5026AE5AAF5B0FBF00010E9070
:100E3E006E0E120048AE5AAF5BE493FC906E0E122B
:100E4E000048E493900088127008ECF0AE5AAF5B45
:100E5E00906E0E120048E493900088127008E0FC29
:100E6E00906E10120048ECFCE493FDECD39D4019FB
:100E7E00906E10120048E493FC906E0E120048E43F
:100E8E0093900088127008ECF0AE5AAF5B742D6F21
:100E9E004E7006755B33755A00AE5AAF5B74022FF7
:100EAE00FF50010E8E5A8F5B785B740126F650044C
:100EBE0018E436F64003020E0022E50C903609F8CF
:100ECE00282873020F8E75E700A232B34008E5B5ED
:100EDE004408F5B58006E5B554F7F5B575E710028B
:100EEE000F8E75E700A232B34008E5B54402F5B5A2
:100EFE008006E5B554FDF5B575E710020F8EA232EA
:100F0E0092A2807CA23292A1807675E700A232B3C3
:100F1E004008E5B54440F5B58006E5B554BFF5B5D6
:100F2E0075E710805B75E700A232B34008E5B54463
:100F3E0080F5B58006E5B5547FF5B575E7108040B0
:100F4E00A2329287803AA2329290803475E700A244
:100F5E0032B34008E5B54410F5B58006E5B554EF5B
:100F6E00F5B575E710801975E700A232B34008E5B4
:100F7E00B54420F5B58006E5B554DFF5B575E71037
:10360900020ED1020ED4020EF0020F0C020F1202AA
:103619000F18020F33020F4E020F54020F5A020FF6
:01362900752B
:100F8E002285F97385FA747E017F00E574126FD79E
:100F9E00E5732FFF50010E8E5A8F5BAC5CAD5DEF8B
:100FAE002DFDEE3CFC8C5C8D5D12025B1202661216
:100FBE00027112027C9000D0E0B4032C75A710854C
:100FCE00F97385FA747E017F00E574126FD7E573AD
:100FDE002FFF50010E8E5A8F5B1202871202921251
:100FEE00029D1202AC75A7002275A71085F97385B4
:100FFE00FA747E017F00E574126FD7E5732FFF50F0
:10100E00010E8E5A8F5B7E017F7690010DE0126F7E
:10101E00D7AC5AAD5BED2FFFEC3EFE8E5C8F5DE5DF
:10102E005DF5FDE55CF5FE900078E4F075A70074C3
:10103E001290005DF02285F97385FA747E017F00AF
:10104E00E574126FD7E5732FFF50010E8E5A8F5B2A
:10105E00900019E0FCA3E0FDEF2DFDEE3CFC8C5C56
:10106E008D5DE55DF5FDE55CF5FE220564229000E3
:10107E00D0E0640360079000EEE0B4021EA2D8B385
:10108E004002C293A2D9B34002C294A2DAB3400284
:10109E00C291A2DBB34002C2928044A2D8B3400AEE
:1010AE00C2939000EEE06002C287A2D9B3400AC29A
:1010BE00949000EEE06002C290A2DAB3400EC291AC
:1010CE009000EEE06006E5B554EFF5B5A2DBB34057
:1010DE000EC2929000EEE06006E5B554DFF5B5A2C3
:1010EE00DCB34030A2965006741990005DF0A295C4
:1010FE005006741990005DF0A2A05006741990006D
:10110E005DF0A2975006741990005DF0C296C295DC
:10111E00C2A0C29775D8402285A77275A7109000FD
:10112E00D0E0640360079000EEE0B40224A2D8B3CE
:10113E004002C287A2D9B34002C290A2DAB34006DF
:10114E00E5B554EFF5B5A2DBB34006E5B554DFF5D2
:10115E00B5A2DCB340089000DCE0900078F075D8C2
:10116E00408572A72290F800E4936406600280FE28
:10117E0075B50075840175A70075FF8075EF069033
:10118E000059E4F075C91075A70F75A1C775A700B2
:10119E0075D90075CE0C75A70F75F1FE75F2FF753A
:1011AE00F30775F47875A4BA75A5FF75A60775AE25
:1011BE000075AFFF75D48175D5FF75D6FF75D7FF56
:1011CE0075A70075A20175A14775F80975D8007548
:1011DE00D90475DA0975DB0975DC0975DD0975DE6B
:1011EE000975D84075A71075D80075D90475DA0938
:1011FE0075DB0975DC0975DD0975DE0975D8407575
:10120E00A70075E60875E71075BC0175BE0475BDBF
:10121E006C75BE0775BDA075BE0875BD0175BC00A9
:10122E0075BB1875BC2075BA0875E88075D1137535
:10123E00A70F75E10575E20075C740120AB47597E0
:10124E0000759780740A126FB77597C0E597542092
:10125E00700280F8758F0275A700D2AF7598007571
:10126E00A90C75A70F75AB4375ADFB75AC1E75A7B5
:10127E001075C91875CA0075CB0075C80475A7001E
:10128E00758912758E04758C00758A00C2A9D28C70
:10129E00758D00758B00D2ABD28E75B62075D94484
:1012AE00C299C22874C8F50975080012373275A79D
:1012BE000FE5FB900067F0E5FA900068F0E5F99015
:1012CE000069F075A70090F800E493F527123851E5
:1012DE0090089BE0D39403500790089BE0B401065E
:1012EE00740090089BF074019000D1F090089BE080
:1012FE0090362AF8282873802A802875A70F75F350
:10130E000F75A700A2A3400674029000D1F08013BF
:10131E0075A70F75F31775A700A2A4400674029067
:03132E0000D1F0FB
:0C362A0002130502130702130902131E0D
:101331009000D1E0B4022AC227123BF0740290005F
:10134100D1F090089BE0903636F828287380108001
:0F1351000E74009000E0F0800674009000EDF044
:0C36360002134E02135002135202135AEA
:101360008028D227123B0F74019000D1F090089B87
:10137000E0903642F82828738010800E74009000A8
:0A138000E0F0800674009000EDF02C
:0C36420002137802137A02137C02138436
:10138A0012009E9000DBE07006740A9000DBF09079
:10139A0000BCE0700674E39000BCF09000C2E00468
:1013AA0090007BF012035290F807E49390006EF0DD
:1013BA0090006EE0440A90006EF090006EE054FED9
:1013CA0090006EF0740690005FF07401900060F077
:1013DA0090F802E493900061F07403900062F07454
:1013EA0005900063F0741F900064F0740690006525
:1013FA00F0900061E0B404067404900065F0900077
:10140A0061E0B405067405900065F0740690006604
:10141A00F090F804E49390006AF0740090006BF086
:10142A0090F805E49390006CF090F806E49390002D
:10143A006DF074FF90006FF0120B9F900061E0B4A2
:10144A000505120D2C8011900061E0D3940540052A
:10145A00120C5E8003120DFA9000F7E0900074F00F
:10146A009000AEE0900075F09000AFE0900076F04A
:10147A00A2B6B39204A2B3B39205A2A4B39221A2D4
:10148A00A3B39222900070E4F0756F00743A90074B
:10149A0088F074FD900789F0900071E4F0756E0190
:1014AA0090005DE4F09000D2E0B40106741A900056
:1014BA005DF0C220756300C209D20AC202757100CA
:1014CA00C2231236D8755F00756B007561007565A9
:1014DA0032756600756700756800756900756A007F
:1014EA0090001FE4F0A3F0756C00D2B2D2A4D2B07F
:1014FA00D2B1D2A3D2A7D2A6D2A5D2B7900094E0F5
:10150A00D394FA400674FA900094F07E017F00901A
:10151A000076E0126FD7900075E02FFF50010E9011
:10152A000029EEF0A3EFF0EFD394FFEE940F4007FB
:10153A00900029E4F0A3F0900074E0700674FF9024
:10154A000074F09000D2E07005756D028003756D2D
:10155A00039000D3E0D39401400674009000D3F0C6
:10156A009000D9E0C3940A5006740A9000D9F0900A
:10157A0000E3E0700674019000E3F09000E3E0B449
:10158A00FF0674FE9000E3F09000EAE0D394FE4078
:10159A000674FE9000EAF0900110E0D3940240062F
:1015AA007401900110F0900126E0D3940140067472
:1015BA0001900126F074019000F0F074019000F19E
:1015CA00F074009000F8F07400900118F0D29C902A
:1015DA0000C3E0D39404400674049000C3F0900062
:1015EA00F5E0D39404400674049000F5F0E570D356
:1015FA00941040037570109006CFE0D3940C400607
:10160A0074009006CFF09006D3E0D3940C40067491
:10161A00009006D3F09006D7E0D3940C40067400ED
:10162A009006D7F09006DBE0D3940C400674009045
:10163A0006DBF09006DFE0D3940C400674009006B7
:10164A00DFF09006E3E0D3940C400674009006E3C2
:10165A00F09006E7E0D3940C400674009006E7F099
:10166A009006EBE0D3940C400674009006EBF090E1
:10167A0006EFE0D3940C400674009006EFF0900653
:10168A00F3E0D3940C400674009006F3F0D2EC75A4
:10169A00CF01A298B34005C298123CD1E54D60062D
:1016AA00A299B3B340028005C2991241B2E54E64D1
:1016BA00016005E54EB4040280D5C28E7E107F001B
:1016CA00E564126FD7E58D75F010A4FDACF0EF2D2F
:1016DA00FDEE3CFCE58B75F01084FF7E00ED2FFFDC
:1016EA00EC3EFE8E548F55D28E9000B5E060099084
:1016FA0000B5E0C3943D4002805C900021126FE582
:10170A00900021E0FEA3E0FF900023E0FCA3E0FDAF
:10171A00EFB50542EEB5043EB217A203B340197500
:10172A00E700A217B34008E5B54404F5B58006E51D
:10173A00B554FBF5B575E710900023E0FEA3E0FF72
:10174A00900025E0FCA3E0FDEF2DFDEE3CFC9000AF
:10175A0023ECF0A3EDF09000C2E060099000C2E033
:10176A00C3940340030217FD125D7FA203B350091D
:10177A00900070E0C3942B400280069000ACE0F524
:10178A0045E54575F002A4FFAEF0900890EEF0A38F
:10179A00EFF0900099E0C395614007E55FC395605B
:1017AA005007900890E4F0A3F075E700AE2EAF2F33
:1017BA00900890E0FCA3E0FDEFD39DEE9C4015E578
:1017CA00B554F7F5B59000C2E0B40206E5B5440297
:1017DA00F5B5801C900070E0C394415013E5B54400
:1017EA0008F5B59000C2E0B40206E5B554FDF5B5BA
:1017FA0075E7109000C2E0B4032A125E9A75E700FA
:10180A00AE2EAF2F900890E0FCA3E0FDEFD39DEE43
:10181A009C4008E5B54408F5B58006E5B554F7F5EA
:10182A00B575E71090009DE06009A2B3300501B3D9
:10183A00B340028056A2B3300501B3404EA2B33082
:10184A000701B34039A21B4030900082E0D3955E75
:10185A004025900084E07013900083E0B401069064
:10186A0000847401F0900083E004F0A21AB34005EA
:10187A00900083E4F0D21AD21BA207B39205A20702
:10188A00B330B301B34004A2079205A2B6300401F3
:10189A00B35003021F5BA2B6300401B35003021F08
:1018AA005BA2B6300601B35003021E07756E0090A4
:1018BA0000B5E0B43D1975E700A206B34008E5B5E6
:1018CA0054FBF5B58006E5B54404F5B575E7100592
:1018DA005EA208B3B35013AE54AF55900010E0FCAB
:1018EA00A3E0FDEDC39FEC9E4003021ABEE56DB472
:1018FA00032EA229B34022E55EB43B03756D01E5D0
:10190A005EC3943B500690005D7401F0E55ED3948B
:10191A003B4006740290005DF0755E01D229806238
:10192A00E56DB4020A756D01755E3BC21AC21CE50B
:10193A005EB43B05755E01804990005DE07034E558
:10194A005EC3943B500690005D7401F0E55ED3944B
:10195A003B4006740290005DF0E55EC3943B500282
:10196A00D220E55ED3943B4002D220C296C295C2F1
:10197A00A0C2979000D2E0B40105120AB4800375A0
:10198A005E01AE56AF57AC54AD55EF2DFDEE3CFCA3
:10199A0074028C068D071200398E568F579000B547
:1019AA00E060099000B5E0C3943D40028049900090
:1019BA0021E0FEA3E0FF9000B5E08E048F05FF1240
:1019CA006FC774018C068D07120039900025EEF05E
:1019DA00A3EFF0900025E0F8A3E0900023C8F0A35D
:1019EA00C8F0900021E4F0A3F0C21775E700E5B54E
:1019FA0054FBF5B575E710A2A4B34002C221A2A315
:101A0A00B34002C222A220B34002C220B21D9000FB
:101A1A0084E0B40111A21AB34004D21D8002C21D8F
:101A2A007402900084F0900084E0C394025006A2ED
:101A3A0003B3B3400280067402900084F09000DE83
:101A4A00E0640460079000D0E0B4036290009DE077
:101A5A006006900084E07002800DA21C301A01B367
:101A6A004005900083E4F09000D2E064016006A291
:101A7A0026B3B3501790009DE06009A21A301C01EA
:101A8A00B3B340028006740590005DF0B21CA21B3D
:101A9A00B3401BA21AB34004D21C8002C21C90009D
:101AAA00D2E07006900084E070028002D226C21A48
:101ABA00C21B803AAE56AF57AC54AD55EF2DFDEE72
:101ACA003CFC74018C068D071200398E568F57E53F
:101ADA006DC39402500DAC54AD5574B8C39D740BCC
:101AEA009C40028009120AB4740690005DF0E55E1B
:101AFA00B43B12740390005DF0D2209000D2E0B49F
:101B0A000103120AB4AE58AF59AC54AD55EF2DFDCE
:101B1A00EE3CFC8C588D59AE54AF55EFD39DEE9CDC
:101B2A004011900017E0FAA3E0FBEBC394E8EA94B3
:101B3A000340028006900017126FE5900014E0FE41
:101B4A00A3E0FFAC54AD55EF2DFDEE3CFC90001424
:101B5A00ECF0A3EDF09000D2E0B40118AE54AF550A
:101B6A007405126FD77401120039900010EEF0A3B9
:101B7A00EFF08011AE54AF557402126FD790001077
:101B8A00EEF0A3EFF0C28E758D00758B00756400C0
:101B9A00755501755400D28EE55E240E75F00F84DA
:101BAA00AFF07E00EF4E6003021C37E56D6013AEA6
:101BBA0056AF57740F126FD7900012EEF0A3EFF0E2
:101BCA00800F900014E0F8A3E0900012C8F0A3C8B8
:101BDA00F0900012E0FEA3E0FFEF4E600B7C7B7DED
:101BEA005C126EC58E528F53900014E4F0A3F0AECF
:101BFA0052AF537428BE00039F5010E5632FFF5065
:101C0A00010E74011200398E528F5385536390006E
:101C1A00D9E0A852B8000DD395534008E553900077
:101C2A005CF080099000D9E01490005CF09000D03C
:101C3A00E0B40308900051E0655E6002800EA21DC8
:101C4A00301E01B34004D21F8002C21FE55E640B3E
:101C5A006005E55EB429099000C2E06003125A4BA0
:101C6A0090005AE0655E600790005BE0B55E037520
:101C7A006F00A209B35006A208B3B34003021D2F96
:101C8A0090008EE0B40173900110E0B40214124384
:101C9A0053900079E075F0BEA4FFAEF08E5C8F5DC4
:101CAA008056E56775F00A84FF7E00900588120069
:101CBA0048E0F55B755A00AE5AAF5B9000B3E0128C
:101CCA006FD774648E048F05FF126FC78C5C8D5DAD
:101CDA00E55D900016F0AE5AAF5B90008CE0126F93
:101CEA00D774648E048F05FF126FC774BE8C068D7D
:101CFA0007126FD78E5C8F5D801790008CE075F0AD
:101D0A00BEA4FFAEF08E5C8F5D9000B3E09000162B
:101D1A00F0E561C394CC5006E55D455C7002800332
:101D2A00120F8FD209E56DB40106E55E64116002F7
:101D3A00800C75700190005E7401F0756D00E56DA0
:101D4A006003021E029000D5E0600D900078E0A8C2
:101D5A0052B800069553400280489000D5E0B4027C
:101D6A002790004DE0655E601790004EE0655E606A
:101D7A000F90004FE0655E6007900050E0B55E038B
:101D8A00757003756C00800CC200756C0090001FA2
:101D9A00E4F0A3F0900078E06006740990005DF02A
:101DAA00805690004DE0655E601790004EE0655EDB
:101DBA00600F90004FE0655E6007900050E0B55EEE
:101DCA003775700190004DE0B55E0690005E7401B3
:101DDA00F090004EE0B55E06740290005EF090004E
:101DEA004FE0B55E06740390005EF0900050E0B5D7
:101DFA005E06740490005EF0A206B39204A206B3D3
:101E0A0030B601B35003021F5B756E019000B5E056
:101E1A00B43D1975E700A206B34008E5B54404F5D8
:101E2A00B58006E5B554FBF5B575E710A22840055F
:101E3A0075FFA0D22875E700E5B54401F5B575E749
:101E4A0010742B900070F0A2069204E55ED3944AB7
:101E5A004014D208E55ED39485400B740490005D6B
:101E6A00F0D220755E469000DDE0B40107E56AC352
:101E7A00941440028009120AB4741390005DF0E5CC
:101E8A006AC394415009740E90005DF0120AB4902E
:101E9A000065E0FE900061E0C39E4009900061E0A9
:101EAA00D39408400974FB90005DF0120AB49000C4
:101EBA006AE0601590006AE0FE900064E06E6009D6
:101ECA0074FE90005DF0120AB490089BE0600690E0
:101EDA00010DE06002807A74019000D1F090089BB5
:101EEA00E090364EF828287380188016A2A3400680
:101EFA0074029000D1F0800AA2A4400674029000F5
:021F0A00D1F014
:0C364E00021EF2021EF4021EF6021F0211
:101F0C009000D1E0B40105A227B340028019D2277A
:101F1C00120AB4123B0F74019000D1F012009ED241
:101F2C0023741B90005DF09000D1E0B40206A22750
:101F3C00B3B340028019C227120AB4123BF07402E8
:101F4C009000D1F012009ED223741B90005DF0A281
:101F5C0020B34008C296C295C2A0C29790010DE072
:101F6C00600CAE52AF537414BE00059F4002803714
:101F7C00900095E090365AF8282873802A8028A281
:101F8C00A3B35005A222B340028005120FF7D22250
:101F9C008015A2A4B35005A221B340028005120FF4
:071FAC00F7D2218002800042
:10365A00021F87021F89021F8B021F9E021FB102CF
:02366A001FB38C
:101FB300A20BB3B35008900051E0655E60030221A9
:101FC30037A201B35006A200B3B3400302212F90FE
:101FD30000D0E0B4030280030220F6900084E0B452
:101FE300020280030220C5A21FB340581201FE90D3
:101FF3000121E0601F90001DE0FEA3E0FF900119A6
:10200300E0126FD774C88E048F05FF126FC78C5C04
:102013008D5D800A90001DE0F55CA3E0F55DAE5C8C
:10202300AF5D745E126FD774058E048F05FF126F58
:10203300C7AE5AAF5BED2FFFEC3EFE8E5C8F5D1299
:10204300025B805C12022B900121E0D39404401FB9
:1020530090001DE0FEA3E0FF90011DE0126FD77416
:10206300C88E048F05FF126FC78C5C8D5D800A904C
:10207300001DE0F55CA3E0F55DAE5CAF5D745E1240
:102083006FD774058E048F05FF126FC7AE5AAF5B0F
:10209300ED2FFFEC3EFE8E5C8F5D12028775A7006D
:1020A3009000EEE0B4011975E700A202B34008E521
:1020B300B54480F5B58006E5B5547FF5B575E710F1
:1020C300802F1201FE12025B12022B12028775A7E8
:1020D300009000EEE0B4011975E700A202B34008D6
:1020E300E5B54480F5B58006E5B5547FF5B575E7EC
:1020F3001080399000EEE0C39402500F1201FE12DB
:10210300025BA202B34002D28780211201FE1202B7
:102113005B12022BAE5AAF5BAC2CAD2DEF2DFDEE57
:102123003CFC8C5C8D5D12028775A700C20BD20C40
:10213300D20DD20EA20CB3B35008900052E0655EEC
:1021430060030222BEA201B35006A200B3B3400350
:102153000222B69000D0E0B40302800302227D90F5
:102163000084E0B40202800302224CA21FB3405B4E
:102173001201FE900121E0D39401401F90001DE065
:10218300FEA3E0FF90011AE0126FD774C88E048F8C
:1021930005FF126FC78C5C8D5D800A90001DE0F512
:1021A3005CA3E0F55DAE5CAF5D745E126FD7740542
:1021B3008E048F05FF126FC7AE5AAF5BED2FFFEC96
:1021C3003EFE8E5C8F5D120266805C12022B9001D4
:1021D30021E0D39405401F90001DE0FEA3E0FF9093
:1021E300011EE0126FD774C88E048F05FF126FC7EC
:1021F3008C5C8D5D800A90001DE0F55CA3E0F55DCD
:10220300AE5CAF5D745E126FD774058E048F05FFED
:10221300126FC7AE5AAF5BED2FFFEC3EFE8E5C8FA5
:102223005D12029275A7009000EEE0B4011975E704
:1022330000A202B34008E5B54480F5B58006E5B5D4
:10224300547FF5B575E710802F1201FE1202661256
:10225300022B12029275A7009000EEE0B4011975EB
:10226300E700A202B34008E5B54480F5B58006E572
:10227300B5547FF5B575E71080399000EEE0C3944F
:1022830002500F1201FE120266A202B34002D29064
:1022930080211201FE12026612022BAE5AAF5BAC12
:1022A3002CAD2DEF2DFDEE3CFC8C5C8D5D1202926E
:1022B30075A700D20BC20CD20DD20EA20DB3B35030
:1022C30008900053E0655E6003022449A201B35005
:1022D30006A200B3B340030224419000D0E0B4034C
:1022E300028003022404900084E0B402028003020B
:1022F30023D3A21FB3405B1201FE900121E0D394CC
:1023030003401F90001DE0FEA3E0FF90011BE012BD
:102313006FD774C88E048F05FF126FC78C5C8D5DF9
:10232300800A90001DE0F55CA3E0F55DAE5CAF5D57
:10233300745E126FD774058E048F05FF126FC7AEDC
:102343005AAF5BED2FFFEC3EFE8E5C8F5D12027188
:10235300805C12022B900121E0D39406401F900071
:102363001DE0FEA3E0FF90011FE0126FD774C88E3B
:10237300048F05FF126FC78C5C8D5D800A90001D72
:10238300E0F55CA3E0F55DAE5CAF5D745E126FD704
:1023930074058E048F05FF126FC7AE5AAF5BED2F26
:1023A300FFEC3EFE8E5C8F5D12029D75A7009000D0
:1023B300EEE0B4011975E700A202B34008E5B544A5
:1023C30080F5B58006E5B5547FF5B575E710802F28
:1023D3001201FE12027112022B12029D75A70090C8
:1023E30000EEE0B4011975E700A202B34008E5B5B9
:1023F3004480F5B58006E5B5547FF5B575E71080E3
:102403003D9000EEE0C3940250131201FE120271DC
:10241300A202B34006E5B54410F5B580211201FED2
:1024230012027112022BAE5AAF5BAC2CAD2DEF2D05
:10243300FDEE3CFC8C5C8D5D12029D75A700D20BFA
:10244300D20CC20DD20EA20EB3B35008900054E0CA
:10245300655E60030225D4A201B35006A200B3B3A4
:1024630040030225CC9000D0E0B403028003022590
:102473008F900084E0B40202800302255EA21FB3A2
:10248300405B1201FE900121E0D39403401F9000B2
:102493001DE0FEA3E0FF90011CE0126FD774C88E0D
:1024A300048F05FF126FC78C5C8D5D800A90001D41
:1024B300E0F55CA3E0F55DAE5CAF5D745E126FD7D3
:1024C30074058E048F05FF126FC7AE5AAF5BED2FF5
:1024D300FFEC3EFE8E5C8F5D12027C805C12022B51
:1024E300900121E0D39407401F90001DE0FEA3E07C
:1024F300FF900120E0126FD774C88E048F05FF127E
:102503006FC78C5C8D5D800A90001DE0F55CA3E0D5
:10251300F55DAE5CAF5D745E126FD774058E048F8C
:1025230005FF126FC7AE5AAF5BED2FFFEC3EFE8E79
:102533005C8F5D1202AC75A7009000EEE0B4011948
:1025430075E700A202B34008E5B54480F5B58006FF
:10255300E5B5547FF5B575E710802F1201FE120221
:102563007C12022B1202AC75A7009000EEE0B401BE
:102573001975E700A202B34008E5B54480F5B580BC
:1025830006E5B5547FF5B575E710803D9000EEE0A4
:10259300C3940250131201FE12027CA202B340063E
:1025A300E5B54420F5B580211201FE12027C12022A
:1025B3002BAE5AAF5BAC2CAD2DEF2DFDEE3CFC8C5E
:1025C3005C8D5D1202AC75A700D20BD20CD20DC28A
:1025D3000EE57090366CF8282873022B9E9000F558
:0125E300E017
:06366C000225DD0225E04D
:1025E4009036ABF82828731253ED80121253ED8005
:0E25F4000D12547780081255238003125523D0
:0F36AB000225EB0225F00225F50225FA0225FF84
:10260200757002022B9E12564F125766125A809014
:102612000888E0FEA3E0FF740A126FD7900012E070
:10262200FCA3E0FD74098F02FF126FC78D078C03B4
:102632008E048A058B06126EC590088CEEF0A3EF0D
:10264200F09000DEE0B40108743CBE00059F400239
:10265200800D743C90088CF8E4F0E8A3F0801B90A5
:10266200088CE0FEA3E0FF74F0BE00039F500B74E1
:10267200F090088CF8E4F0E8A3F0E53670037536C4
:102682000190088CE0FEA3E0FFE5362FFF50010E1B
:0F26920090088CEEF0A3EFF075700390005EE0FF
:0336720002260825
:1026A1009036BAF82828738022A231400375700A47
:1026B1008019A231400375700B8010A2314003755F
:0B26C100700C8007A231400375700D03
:0F36BA000226A80226AA0226B30226BC0226C5B3
:1026CC00022B9E9006CFE06006750801125BA79066
:1026DC00010EE0B4011490010FE0A852B80004956B
:1026EC00535007E55FC39560400280097415900054
:1026FC005DF00227829000C3E0D39402403F90002B
:10270C0097E02403A852B8000495535009900099FF
:10271C00E0D3956150028008D201740890005DF0FE
:10272C00900097E0A852B80005D39553500B900039
:10273C0099E02403C395615002C20180399000973F
:10274C00E02403A852B8000495535007E55FC395E5
:10275C006040028008D201740890005DF0900097F0
:10276C00E0A852B80005D395535009E560240FC377
:10277C00955F5002C2019000DDE07007E56AC394DA
:10278C001440028002D2019000D2E0B40102D201C6
:10279C00A2014005757004800A75701090001FE44A
:0A27AC00F0A3F0022B9E9000C3E0A2
:063675000226CF0227B27D
:1027B6009036C9F828287312443D801212443D8091
:0E27C6000D1245EB800812469D800312469DC1
:0F36C9000227BD0227C20227C70227CC0227D142
:1027D4009006D3E06006750802125BA775700502C7
:1027E4002B9E1247DD7570069006D7E060067508CB
:1027F40003125BA79006DBE06006750804125BA772
:10280400022B9E900016E06006A203B3B340028040
:102814001D900016E02529FFAE2850010E8E288F4A
:1028240029E55ED3940F5006900016E014F0124A86
:10283400237570079006DFE06006750805125BA734
:102844009006E3E06006750806125BA7022B9E90D3
:102854000110E0B402031243CB124E53757008907A
:1028640006E7E06006750807125BA79006EBE060D8
:1028740006750808125BA7022B9E12520FA20BB317
:102884005005A20CB340028008D20BD20CD20DD258
:102894000E7570109006EFE06006750809125BA7CC
:1028A4009006F3E0600675080A125BA7022B9E02ED
:1028B4002B9E90003FE0C394465008C29674469005
:1028C400003FF0900055E0B4011DE5362406F536CE
:1028D40090088CE0FEA3E0FF74062FFF50010E90D9
:1028E400088CEEF0A3EFF0900055E0B4021DE5363D
:1028F400240CF53690088CE0FEA3E0FF740C2FFF47
:1029040050010E90088CEEF0A3EFF085365B755AFB
:102914000090004DE0F5731202BBE55D90003FF0BE
:10292400900008E55AF0A3E55BF0E573900040F0F1
:10293400C21090088CE0F55AA3E0F55B90004DE0DE
:10294400F5731202BBE55D90003DF0900000E55A7E
:10295400F0A3E55BF0E57390003EF0C20F757003E1
:10296400022B9E900043E0C3944650139000DEE097
:10297400B40104C2968002C2957446900043F0905C
:102984000056E0B4011DE5362406F53690088CE0C7
:10299400FEA3E0FF74062FFF50010E90088CEEF0AA
:1029A400A3EFF0900056E0B4021DE536240CF53692
:1029B40090088CE0FEA3E0FF740C2FFF50010E90F2
:1029C400088CEEF0A3EFF085365B755A0090004E4C
:1029D400E0F5731202BBE55D900043F090000AE558
:1029E4005AF0A3E55BF0E573900044F0C21290083E
:1029F4008CE0F55AA3E0F55B90004EE0F57312020B
:102A0400BBE55D900041F0900002E55AF0A3E55B60
:102A1400F0E573900042F0C211757003022B9E9092
:102A24000047E0C3944650139000DEE0B40104C2B2
:102A3400968002C2A07446900047F0900057E0B41C
:102A4400011DE5362406F53690088CE0FEA3E0FF70
:102A540074062FFF50010E90088CEEF0A3EFF09057
:102A64000057E0B4021DE536240CF53690088CE0DE
:102A7400FEA3E0FF740C2FFF50010E90088CEEF0C3
:102A8400A3EFF085365B755A0090004FE0F57312A2
:102A940002BBE55D900047F090000CE55AF0A3E519
:102AA4005BF0E573900048F0C21490088CE0F55A8E
:102AB400A3E0F55B90004FE0F5731202BBE55D9077
:102AC4000045F0900004E55AF0A3E55BF0E573904F
:102AD4000046F0C213757003022B9E90004BE0C3B6
:102AE400944650139000DEE0B40104C2968002C202
:102AF40097744690004BF0900058E0B4011DE53601
:102B04002406F53690088CE0FEA3E0FF74062FFF40
:102B140050010E90088CEEF0A3EFF0900058E0B452
:102B2400021DE536240CF53690088CE0FEA3E0FF88
:102B3400740C2FFF50010E90088CEEF0A3EFF0857B
:102B4400365B755A00900050E0F5731202BBE55DE8
:102B540090004BF090000EE55AF0A3E55BF0E573AE
:102B640090004CF0C21690088CE0F55AA3E0F55B97
:102B7400900050E0F5731202BBE55D900049F090BF
:102B84000006E55AF0A3E55BF0E57390004AF0C255
:0A2B940015757003800480028000B4
:10367B000227E602280702285302287E0228B302FB
:10368B0028B6022967022A23022ADF022B9A022B71
:04369B009C022B9EC4
:102B9E0090003DE0B55E028003022C40A20F407211
:102BAE00900000E0FEA3E0FFEF4E6021AE56AF575F
:102BBE00900000E0FCA3E0FD12000374068E048F6B
:102BCE0005FF126FC7900000ECF0A3EDF090003EF1
:102BDE00E0601A900000E0FEA3E0FFAC56AD57EFA8
:102BEE002DFDEE3CFC900000ECF0A3EDF090003ECD
:102BFE00E0D39401401A900000E0FEA3E0FFAC5633
:102C0E00AD57EF2DFDEE3CFC900000ECF0A3EDF087
:102C1E00D20FAE54AF55900000E0FCA3E0FDEFC321
:102C2E009DEE9C400D121044D296C20F74C89000B7
:102C3E003DF0A20FB3B3500790003DE0B55E0280A9
:102C4E000D121044D29674C890003DF0C20F900041
:102C5E003FE0B55E028003022CFBA2104072900092
:102C6E0008E0FEA3E0FFEF4E6021AE56AF57900096
:102C7E0008E0FCA3E0FD12000374068E048F05FF2E
:102C8E00126FC7900008ECF0A3EDF0900040E060EA
:102C9E001A900008E0FEA3E0FFAC56AD57EF2DFDF5
:102CAE00EE3CFC900008ECF0A3EDF0900040E0D379
:102CBE009401401A900008E0FEA3E0FFAC56AD5719
:102CCE00EF2DFDEE3CFC900008ECF0A3EDF0D210E1
:102CDE00AE54AF55900008E0FCA3E0FDEFC39DEEAF
:102CEE009C400AC296744690003FF0C210A210B3E8
:102CFE00B3500790003FE0B55E02800AC29674465C
:102D0E0090003FF0C210900041E0B55E02800302D9
:102D1E002DC1A2114072900002E0FEA3E0FFEF4E23
:102D2E006021AE56AF57900002E0FCA3E0FD12000A
:102D3E000374068E048F05FF126FC7900002ECF02D
:102D4E00A3EDF0900042E0601A900002E0FEA3E0D6
:102D5E00FFAC56AD57EF2DFDEE3CFC900002ECF0B3
:102D6E00A3EDF0900042E0D39401401A900002E0EF
:102D7E00FEA3E0FFAC56AD57EF2DFDEE3CFC9000F0
:102D8E0002ECF0A3EDF0D211AE54AF55900002E07C
:102D9E00FCA3E0FDEFC39DEE9C4018121044900082
:102DAE00DEE0B40104D2968002D295C21174C890AE
:102DBE000041F0A211B3B35007900041E0B55E029E
:102DCE0080181210449000DEE0B40104D296800206
:102DDE00D29574C8900041F0C211900043E0B55EE8
:102DEE00028003022E92A212407290000AE0FEA30D
:102DFE00E0FFEF4E6021AE56AF5790000AE0FCA305
:102E0E00E0FD12000374068E048F05FF126FC7904B
:102E1E00000AECF0A3EDF0900044E0601A90000A76
:102E2E00E0FEA3E0FFAC56AD57EF2DFDEE3CFC905F
:102E3E00000AECF0A3EDF0900044E0D39401401AA8
:102E4E0090000AE0FEA3E0FFAC56AD57EF2DFDEE6D
:102E5E003CFC90000AECF0A3EDF0D212AE54AF554C
:102E6E0090000AE0FCA3E0FDEFC39DEE9C401590A0
:102E7E0000DEE0B40104C2968002C2957446900052
:102E8E0043F0C212A212B3B35007900043E0B55EF6
:102E9E000280159000DEE0B40104C2968002C29555
:102EAE007446900043F0C212900045E0B55E028079
:102EBE0003022F63A2134072900004E0FEA3E0FF12
:102ECE00EF4E6021AE56AF57900004E0FCA3E0FD3C
:102EDE0012000374068E048F05FF126FC790000454
:102EEE00ECF0A3EDF0900046E0601A900004E0FED6
:102EFE00A3E0FFAC56AD57EF2DFDEE3CFC90000469
:102F0E00ECF0A3EDF0900046E0D39401401A90004F
:102F1E0004E0FEA3E0FFAC56AD57EF2DFDEE3CFCFA
:102F2E00900004ECF0A3EDF0D213AE54AF55900028
:102F3E0004E0FCA3E0FDEFC39DEE9C40181210448C
:102F4E009000DEE0B40104D2968002D2A0C21374C7
:102F5E00C8900045F0A213B3B35007900045E0B5FA
:102F6E005E0280181210449000DEE0B40104D29686
:102F7E008002D2A074C8900045F0C213900047E0C2
:102F8E00B55E028003023034A214407290000CE051
:102F9E00FEA3E0FFEF4E6021AE56AF5790000CE05F
:102FAE00FCA3E0FD12000374068E048F05FF126F62
:102FBE00C790000CECF0A3EDF0900048E0601A9082
:102FCE00000CE0FEA3E0FFAC56AD57EF2DFDEE3C3E
:102FDE00FC90000CECF0A3EDF0900048E0D39401CF
:102FEE00401A90000CE0FEA3E0FFAC56AD57EF2D5B
:102FFE00FDEE3CFC90000CECF0A3EDF0D214AE54C0
:10300E00AF5590000CE0FCA3E0FDEFC39DEE9C409D
:10301E00159000DEE0B40104C2968002C2A0744690
:10302E00900047F0C214A214B3B35007900047E0CB
:10303E00B55E0280159000DEE0B40104C2968002F7
:10304E00C2A07446900047F0C214900049E0B55EED
:10305E00028003023105A2154072900006E0FEA325
:10306E00E0FFEF4E6021AE56AF57900006E0FCA396
:10307E00E0FD12000374068E048F05FF126FC790D9
:10308E000006ECF0A3EDF090004AE0601A90000606
:10309E00E0FEA3E0FFAC56AD57EF2DFDEE3CFC90ED
:1030AE000006ECF0A3EDF090004AE0D39401401A34
:1030BE00900006E0FEA3E0FFAC56AD57EF2DFDEEFF
:1030CE003CFC900006ECF0A3EDF0D215AE54AF55DB
:1030DE00900006E0FCA3E0FDEFC39DEE9C401812AD
:1030EE0010449000DEE0B40104D2968002D297C262
:1030FE001574C8900049F0A215B3B350079000495B
:10310E00E0B55E0280181210449000DEE0B40104B7
:10311E00D2968002D29774C8900049F0C2159000E2
:10312E004BE0B55E0280030231D6A21640729000CB
:10313E000EE0FEA3E0FFEF4E6021AE56AF579000BB
:10314E000EE0FCA3E0FD12000374068E048F05FF53
:10315E00126FC790000EECF0A3EDF090004CE06003
:10316E001A90000EE0FEA3E0FFAC56AD57EF2DFD1A
:10317E00EE3CFC90000EECF0A3EDF090004CE0D392
:10318E009401401A90000EE0FEA3E0FFAC56AD573E
:10319E00EF2DFDEE3CFC90000EECF0A3EDF0D21600
:1031AE00AE54AF5590000EE0FCA3E0FDEFC39DEED4
:1031BE009C40159000DEE0B40104C2968002C297D6
:1031CE00744690004BF0C216A216B3B3500790008F
:1031DE004BE0B55E0280159000DEE0B40104C296AD
:1031EE008002C297744690004BF0C2169000E0E049
:1031FE00B40202800302332E900072E0D395665023
:10320E0064900072E0F4042566FE9000E3E08E0008
:10321E00F5F0E884FF7E008F73EFC39410500CEF2F
:10322E008573F0A4FDACF08D7380037573FF900071
:10323E0072E0D39573400B900072E0C39573F571F5
:10324E0080037571009000FEE0D3957140069000EA
:10325E00FEE0F5719000FFE0C3957150069000FFFF
:10326E00E0F5718071900072E0C39566FE9000E308
:10327E00E08E00F5F0E884FF7E008F73EFC39410AC
:10328E00500CEF8573F0A4FDACF08D738003757355
:10329E00FF85735B755A00900072E0255BFFAE5A96
:1032AE0050010E8E5A8F5B74FFBE0009D39F4005EE
:1032BE00855B7180037571FF9000FEE0D3957140C0
:1032CE00069000FEE0F5719000FFE0C39571500688
:1032DE009000FFE0F571A203B3B3500D900073E0C0
:1032EE00FE9000EBE0D39E50028014740790005DB8
:1032FE00F075E700E5B554BFF5B575E7108021759B
:10330E00A71075E700E5CDC395714008E5B554BF2C
:10331E00F5B58006E5B54440F5B575E71075A7001F
:10332E009000FBE0604E900105E0A852B8000495B5
:10333E00535017900104E0A852B8000ED395534095
:10334E0009900106E0D395614002801575A710E53E
:10335E00CDC394BF4004C2A28002D2A275A7008042
:10336E001375A710E5CDC394404004C2A28002D2CB
:10337E00A275A7009000FCE0604E900108E0A852F4
:10338E00B8000495535017900107E0A852B8000EEC
:10339E00D395534009900109E0D395614002801501
:1033AE0075A710E5CDC394BF4004C2A18002D2A17F
:1033BE0075A700801375A710E5CDC394404004C2D5
:1033CE00A18002D2A175A700E56FC39409500AA28D
:1033DE00EDB34005C2ED126041AE54AF557410C34B
:1033EE009F74279E400C900071E0C3945A400302D4
:1033FE003606A208B34009120AB4740690005DF0B6
:10340E00A20AB3500EE561D394334007E561C3942D
:10341E00CC4002804A900110E0B402141243539043
:10342E000079E075F050A4FFAEF08E5C8F5D800FDA
:10343E0090008CE075F050A4FFAEF08E5C8F5DE5D1
:10344E005D455C601AA228400575FFA0D228E5B53F
:10345E004401F5B5742B900070F0120F8FD20A90C4
:10346E000071E0D394014007E561C3941A400280D5
:10347E0002C20A9006CFE06006750801125BA790A3
:10348E0006D3E06006750802125BA79006D7E060CF
:10349E0006750803125BA79006DBE060067508044C
:1034AE00125BA79006DFE06006750805125BA79019
:1034BE0006E3E06006750806125BA79006E7E0607B
:1034CE0006750807125BA79006EBE0600675080804
:1034DE00125BA79006EFE06006750809125BA790D5
:1034EE0006F3E0600675080A125BA7900071E0C350
:1034FE00945A5026E56FB40909900071E004F075F6
:10350E006F00900071E0B45A0FA228400575FFA01D
:10351E00D228E5B54401F5B5803BE56FB4090375D6
:10352E006F00755500755400758D00758B007564B0
:10353E0000900070E0C394415008900070E004F0D9
:10354E0080067441900070F0900070E0B44106E582
:10355E00B554FEF5B5900071E0D394014007E56ACD
:10356E00C3944140028009740E90005DF0120AB4BB
:10357E0090089BE0600690010DE06002807A740175
:10358E009000D1F090089BE090369FF82828738029
:10359E00188016A2A3400674029000D1F0800AA2F1
:0935AE00A4400674029000D1F063
:0C369F0002359D02359F0235A10235ADB9
:1035B7009000D1E0B40105A227B340028019D227B9
:1035C700120AB4123B0F74019000D1F012009ED280
:1035D70023741B90005DF09000D1E0B40206A2278F
:1035E700B3B340028019C227120AB4123BF0740227
:1035F7009000D1F012009ED223741B90005DF00260
:02360700169912
:10694A000000010001400160018001A001C001E0D6
:10695A0002000300039603B603D603F404000500FD
:10696A000512052405360548055A056C057E05906D
:10697A0005A805C005DE0600061406280646066EAA
:10698A0006AE05CF00FF013F015F017F019F01BFF6
:10699A0001DF01FF02FF039503B503D503F303FFEC
:1069AA0004FF05110523053505470559056B057DC6
:1069BA00058F05A705BF05CE05F10613062706456F
:1069CA00066D06AD06ED05DD0FAA0FA50F9F0F9AFE
:1069DA000F940F8D0F870F800F780F710F680F605C
:1069EA000F570F4E0F450F3B0F300F250F1A0F0E83
:1069FA000F020EF50EE80EDB0ECC0EBE0EAE0E9F8B
:106A0A000E8E0E7D0E6C0E5A0E470E340E200E0C94
:106A1A000DF70DE20DCB0DB50D9D0D850D6D0D54C8
:106A2A000D3A0D200D050CE90CCE0CB10C940C7628
:106A3A000C580C3A0C1B0BFB0BDB0BBB0B9A0B79A0
:106A4A000B570B350B130AF10ACE0AAB0A870A64F5
:106A5A000A400A1C09F809D409B0098C09670943D4
:106A6A00091F08FB08D608B2088E086A08460823D8
:106A7A0007FF07DC07B9079607730751072F070DAA
:106A8A0006EC06CA06AA068906690649062A060AFD
:106A9A0005EC05CD05B0059205750558053C0520A0
:106AAA00050504EA04CF04B5049C04820469045170
:106ABA0004390422040B03F403DE03C803B2039D62
:106ACA00038903750361034D033B0328031603047B
:106ADA0002F202E102D102C002B002A002910282D5
:106AEA000273026502570249023C022F0222021671
:106AFA00020901FD01F201E601DB01D001C601BB79
:106B0A0001B101A7019D0194018B018201790170F4
:106B1A0001680160015801500148014101390132FF
:106B2A00012B0125011E01180111010B010500FFAE
:106B3A0000FA0FA60FA00F990F920F8B0F840F7CEC
:106B4A000F740F6B0F620F580F4E0F430F380F2C35
:106B5A000F1F0F120F050EF70EE80ED80EC80EB74C
:106B6A000EA50E930E800E6C0E580E420E2C0E15AC
:106B7A000DFD0DE40DCB0DB10D950D790D5D0D3F9C
:106B8A000D200D010CE10CC00C9E0C7C0C590C352F
:106B9A000C100BEA0BC40B9E0B760B4F0B260AFD4F
:106BAA000AD40AAA0A800A550A2A09FF09D409A896
:106BBA00097C0950092508F908CD08A10875084A71
:106BCA00081E07F307C8079D07730749072006F73A
:106BDA0006CE06A6067E06570630060A05E405BF57
:106BEA00059B057705540532051004EF04CE04AE63
:106BFA00048F047104530435041903FD03E203C727
:106C0A0003AD0394037B0363034B0334031E03089E
:106C1A0002F302DE02CA02B602A30291027F026DE9
:106C2A00025C024C023C022C021D020E020001F21E
:106C3A0001E401D701CA01BE01B101A6019A018F7F
:106C4A000185017A01700166015D0153014A014122
:106C5A00013901310129012101190112010B010434
:106C6A0000FD00F700F000EA00E400DE00D900D3DE
:106C7A0000CE00C900C400BF00BA00B500B100AD23
:106C8A0000A800A400A0009C009900950091008E25
:0C6C9A00008A008700840081007E007BDF
:1036D800754700900892E4F0A3F07531007530004A
:1036E800754D00754E00C22CD22E90089BE06002EA
:1036F800D22374FE900894F8E4F0E8A3F074FE90E6
:103708000898F8E4F0E8A3F074FE900896F8E4F05E
:10371800E8A3F0745A9008BAF0745A9008BBF0D233
:103728002FC22AC231C230C22B22750B00750A0083
:10373800AE0AAF0BAC08AD09EDC39FEC9E40167402
:10374800FF126FB775CF01780B740126F650041875
:10375800E436F650DB22C2AF75D904758F0375B70E
:10376800A575B7F190F800E4F0758F0175B7A575E8
:10377800B7F1E52790F800F075B7A575B7F190F89F
:1037880001E4F075B7A575B7F19008AEE090F802BE
:10379800F075B7A575B7F19008B2E090F803F07529
:1037A800B7A575B7F19008AFE090F804F075B7A524
:1037B80075B7F19008B0E090F805F075B7A575B742
:1037C800F19008B1E090F806F075B7A575B7F190DB
:1037D80008B3E090F807F0758F0075D944D2AF228E
:1037E800900059E0B4AB61C2AF75D90475B62275C3
:1037F800F522758F0375B7A575B7F1740090F600BB
:10380800F0758F01755B00755A00AE5AAF5B741383
:10381800BE00279F402475B7A575B7F190089A1286
:103828000048E0FC90F600120048ECF0785B740168
:1038380026F6500418E436F650D0758F0075F51149
:1038480075B62075D944D2AF22C2AF75F52275D9A5
:1038580004755B00755A00AE5AAF5B7413BE002244
:103868009F401F90F600120048E493FC90089A12BB
:103878000048ECF0785B740126F6500418E436F63C
:1038880050D575D94475F511D2AF22900059E0B4DE
:10389800AA0280030239D0C2AF75D90475B6227561
:1038A800F522758F0375B7A575B7F1740090EE0012
:1038B800F075B7A575B7F1740090F000F075B7A56D
:1038C80075B7F1740090F200F075B7A575B7F1748B
:1038D8000090F400F0758F01755B00755A00AE5AC0
:1038E800AF5B74FFC39F74019E402475B7A575B77D
:1038F800F1900088120048E0FC90EE00120048ECBD
:10390800F0785B740126F6500418E436F650CF754B
:103918005B00755A00AE5AAF5B74FFC39F74019E7B
:10392800402475B7A575B7F1900288120048E0FCED
:1039380090F000120048ECF0785B740126F6500411
:1039480018E436F650CF755B00755A00AE5AAF5B77
:1039580074FFC39F74019E402475B7A575B7F19095
:103968000488120048E0FC90F200120048ECF0785D
:103978005B740126F6500418E436F650CF755B00E8
:10398800755A00AE5AAF5B74FFC39F74019E402402
:1039980075B7A575B7F1900688120048E0FC90F459
:1039A80000120048ECF0785B740126F6500418E425
:1039B80036F650CF758F0075F51175B62075D94458
:1039C800D2AF743A900788F022900059E0B4AA0266
:1039D8008003023B0EC2AF75D90475B62275F52275
:1039E800758F0375B7A575B7F1740090E600F0758B
:1039F800B7A575B7F1740090E800F075B7A575B76D
:103A0800F1740090EA00F075B7A575B7F1740090ED
:103A1800EC00F0758F01755B00755A00AE5AAF5B0C
:103A280074FFC39F74019E402475B7A575B7F190C4
:103A38000088120048E0FC90E600120048ECF0789C
:103A48005B740126F6500418E436F650CF755B0017
:103A5800755A00AE5AAF5B74FFC39F74019E402431
:103A680075B7A575B7F1900288120048E0FC90E898
:103A780000120048ECF0785B740126F6500418E454
:103A880036F650CF755B00755A00AE5AAF5B74FFBF
:103A9800C39F74019E402475B7A575B7F19004883B
:103AA800120048E0FC90EA00120048ECF0785B74E1
:103AB8000126F6500418E436F650CF755B00755AA7
:103AC80000AE5AAF5B74FFC39F74019E402475B764
:103AD800A575B7F1900688120048E0FC90EC00123A
:103AE8000048ECF0785B740126F6500418E436F6CA
:103AF80050CF758F0075F51175B62075D944D2AFC2
:103B0800743A900788F022C2AF75D90475F522750A
:103B18005B00755A00AE5AAF5B74FFC39F74019E79
:103B2800401F90EE00120048E493FC9000881200B9
:103B380048ECF0785B740126F6500418E436F65029
:103B4800D4755B00755A00AE5AAF5B74FFC39F749F
:103B5800019E401F90F000120048E493FC900288F8
:103B6800120048ECF0785B740126F6500418E4362D
:103B7800F650D4755B00755A00AE5AAF5B74FFC33C
:103B88009F74019E401F90F200120048E493FC903D
:103B98000488120048ECF0785B740126F65004188B
:103BA800E436F650D4755B00755A00AE5AAF5B74B4
:103BB800FFC39F74019E401F90F400120048E493D5
:103BC800FC900688120048ECF0785B740126F650E9
:103BD8000418E436F650D475F51175D944D2AF748B
:103BE8003A900788F0C22D22C2AF75D90475F52224
:103BF800755B00755A00AE5AAF5B74FFC39F7401C2
:103C08009E401F90E600120048E493FC9000881242
:103C18000048ECF0785B740126F6500418E436F698
:103C280050D4755B00755A00AE5AAF5B74FFC39FE2
:103C380074019E401F90E800120048E493FC900233
:103C480088120048ECF0785B740126F6500418E4FA
:103C580036F650D4755B00755A00AE5AAF5B74FFE8
:103C6800C39F74019E401F90EA00120048E493FC31
:103C7800900488120048ECF0785B740126F6500432
:103C880018E436F650D4755B00755A00AE5AAF5B2F
:103C980074FFC39F74019E401F90EC00120048E41B
:103CA80093FC900688120048ECF0785B740126F6C5
:103CB800500418E436F650D475F51175D944D2AFCE
:103CC800743A900788F0D22D22E54E64046006E528
:103CD8009964FF60028031A22C4004D22C8027E531
:103CE8004E600874E6254E90005DF0E54D6008745E
:103CF800F0254D90005DF0E54EB4010280FE754E52
:103D080000754D00C22C8002C22CE54E9068BAF8AE
:103D1800282873754E00E599B4FF03754D01E599A0
:103D2800B4FE03754D02E599B4FD03754D03E5999D
:103D3800B4FC03754D04E599B4FA03754D05E5998E
:103D4800B4FB06754E01120AB4E599B4F906754E2E
:103D580004120AB4E599D394E54007E599C394F0B1
:103D68004002801685994F754E027E017F00E54F0F
:103D7800C394E6126FD78E328F33900892E4F0A383
:103D8800F0E599D394C44007E599C394E6400280CE
:103D98002885994F754E0374E5C3954FF5337532F1
:103DA80000AE32AF3390694A126FA6E493F87401FB
:103DB80093900892C8F0A3C8F0D2990241B1900834
:103DC8009AE0700AA224B35005A225B340028042AB
:103DD800900892E0FEA3E0FF74FFBE00039F500925
:103DE800EFC39446EE94064011900892E0FEA3E0DB
:103DF800FFEFD3946DEE94064013900892E0FEA373
:103E0800E0FF900088120048E599F08003859974D6
:103E18008011900892E0FEA3E0FF9000881200480D
:103E2800E599F0900892126FE5900892E0FEA3E001
:103E3800FFEFB40106EEB407028003023FAA900721
:103E480088E0B43C028003023FAAA224B35005A232
:103E580025B34003023F21C29C90089AE0900126B6
:103E6800F090089BE0900095F090089CE09000B5D9
:103E7800F090089DE09000DEF090089EE090008AA7
:103E8800F090089FE09000D0F09008A0E09000EE3D
:103E9800F09008A1E09000C2F09008A2E09000E045
:103EA800F09008A3E0900110F09008A4E09001744D
:103EB800F09008A5E0900175F09008A6E0900176D2
:103EC800F0120352900074E09000F7F0900075E053
:103ED8009000AEF0900076E09000AFF074AB9000E8
:103EE80059F01237E874AA900059F0A22DB3400592
:103EF8001239D18003123893900059E4F09001747C
:103F0800E0700C900175E07006900176E060028028
:103F180004C2248002D224807EC29C900126E090B4
:103F2800089AF0900095E090089BF09000B5E0901A
:103F3800089CF09000DEE090089DF090008AE090E8
:103F4800089EF09000D0E090089FF09000EEE0907E
:103F580008A0F09000C2E09008A1F09000E0E09086
:103F680008A2F0900110E09008A3F074009008A453
:103F7800F074009008A5F074009008A6F074AB9057
:103F88000059F01237E874AA900059F012389312C9
:103F980039D17599FB80FED29C754E00754D007520
:103FA80099FB0241B1900892E0FEA3E0FFEF4E704A
:103FB80006859931753000900892E0FEA3E0FF7401
:103FC800016F4E701BAC30AD31AA32AB33ED2BFB19
:103FD800EC3AFA8A068B07900088120048E599F0B7
:103FE800900892126FE5900892E0FEA3E0FF740239
:103FF8006F4E7021AC30AD3174566D4C7006E54F84
:1040080064E660028003120AB4120352854F997560
:104018004E00754D000241B1900892E0FEA3E0FF0A
:10402800900088120048E599F0900892126FE59088
:104038000892E0FEA3E0FFAC32AD338F028E038C12
:10404800068D0790698E126FA6E493F9740193FEAA
:10405800EAD39EEB994009854F99754E00754D003E
:104068000241B1900892E0FEA3E0FF9000881200A0
:1040780048E599F0900892126FE5900892E0FEA347
:10408800E0FFEFB40006EEB4010280030241B190F4
:104098000069E0D394C7400B900069E0C394C8F569
:1040A80050801A900069E0D39463400B900069E057
:1040B800C39464F5508006900069E0F550E55075AA
:1040C800F002A4FFAEF08F73EF900088127008EF33
:1040D800FCE0FDEC90008B127008EDFCE0FDEC2D8F
:1040E800B5500280030241A20FEF900088127008B9
:1040F800E573FFE0FCEF90008C127008ECFFE0FC29
:10410800EFC39CB5500280030241A2E57390008A78
:10411800127008E573FFE0FCEF90008D127008EC58
:10412800FFE0FCEF2CB55072E57390008E1270081A
:10413800E0C395509008AEF0E57390008F127008B8
:10414800E0C395509008AFF0E573900092127008A4
:10415800E0C395509008B0F0E57390009312700892
:10416800E0C395509008B1F0E57390009412700880
:10417800E0C395509008B2F0E5739000951270086E
:10418800E0C395509008B3F012375E7599F97464DE
:10419800F50975080012373280FE7599FF7464F5C9
:0941A8000975080012373280FE8F
:0F68BA00023D1B023DC6023FAD02402002406B73
:1041B10022E54D9068C9F82828730242969008922A
:1041C100E0FEA3E0FF90005F120048E0F59990083F
:1041D10092126FE5900892E0FEA3E0FF74116F4E1A
:1041E1007003754D00024296856E990242969008C1
:1041F10092E0FEA3E0FF900088120048E0F599EFFD
:10420100B40107EEB40703754D00900892126FE5F3
:07421100024296900893E0C1
:0F68C9000241BB0241BE0241E90241EF0242140B
:1042180090691DF82828738553998067855F998070
:1042280062856199805D8565998058856799805315
:10423800856899804E8569998049856A99804490F6
:104248000020E0F599803CA22EB340077599FAC288
:104258002E8017A223B3400575990F800B90005D3F
:10426800E0F59990005DE4F0C2238017856B998092
:1042780012856699800D856C9980087599FC800374
:03428800754D0071
:10691D0002421F02422402422902422E0242330247
:10692D00423802423D02424202424702424F024277
:0D693D007402427902427E024283024288C7
:0B428B00900892126FE5800312017B87
:0368D800024293E6
:1042960022E537255BFFAE5A50010E9000881200CA
:1042A60048E0F538E537255BFFAE5A50010E0FBFE3
:1042B60000010E900088120048E0F539853F3BE585
:1042C60038B539058538378041E539D39538401DED
:1042D600E539C39538853AF0A4FFAEF0E53B8E0488
:1042E6008F05FF126FC7ED2538F537801DE538C3FA
:1042F6009539853AF0A4FFAEF0E53B8E048F05FFB5
:10430600126FC7EDF4042538F53722E539D3953811
:10431600401DE539C39538853AF0A4FFAEF0E53B7C
:104326008E048F05FF126FC7ED2538F537801DE522
:1043360038C39539853AF0A4FFAEF0E53B8E048F7D
:1043460005FF126FC7EDF4042538F5372290008E6D
:10435600E0B40170E56775F00A84FF7E008F37E5EB
:104366006775F00A84ADF07C008D3A753F0A755A80
:1043760005755B24E537C3941150051242978006F4
:104386009005BDE0F537E537900079F0E56775F003
:104396000A84FF7E008F37E56775F00A84ADF07CEE
:1043A600008D3A753F0A755A05755B5AE537C39411
:1043B60011500512429780069005F3E0F537E53770
:1043C600900016F02290008EE0B4016AE56775F061
:1043D6000A84FF7E008F37E56775F00A84ADF07CAE
:1043E600008D3A753F0A755A05755B36E537C394F5
:1043F60011500512429780069005CFE0F5378537B4
:104406004BE56775F00A84FF7E008F37E56775F028
:104416000A84ADF07C008D3A753F0A755A05755BC6
:1044260048E537C39411500512429780069005E17E
:10443600E0F53785374C22E55F75F00484FF7E0092
:104446008F37E55F75F00484ADF07C008D3A753FDB
:1044560004755A01755B00E537C3943F5005124257
:104466009780069001C7E0F53785372975280090B3
:10447600005CE075F020A4FFAEF09000D9E08E0459
:104486008F05FF126FC78D379000C1E0D3955F503F
:10449600030245439000E5E0D3955F4010ED90019F
:1044A600C8127008E0F52B752A000245409000B04E
:1044B600E0D3955F4043E5379001C8127008E0F5F8
:1044C60038E5379001E8127008E0F5399000E5E02C
:1044D600F404255FF53A9000B0E0FE9000E5E0F4C4
:1044E600042EF53BE538B539058538378003124388
:1044F6001185372B752A008041E5379001E8127047
:1045060008E0F538E537900208127008E0F53990B2
:1045160000B0E0F404255FF53A9000C1E0FE90009B
:10452600B0E0F4042EF53BE538B53905853837801B
:104536000312431185372B752A000245EA9000E8DD
:10454600E0D3955F5011E537900248127008E0F508
:104556002B752A000245EA9000B1E0D3955F5043DF
:10456600E537900228127008E0F538E537900248E2
:10457600127008E0F5399000B1E0F404255FF53AD1
:104586009000E8E0FE9000B1E0F4042EF53BE5383B
:10459600B53905853837800312431185372B752ABF
:1045A600008041E537900208127008E0F538E537DB
:1045B600900228127008E0F5399000C1E0F4042555
:1045C6005FF53A9000B1E0FE9000C1E0F4042EF5EC
:1045D6003BE538B5390585383780031243118537F1
:1045E6002B752A00229000F9E0F53C753F11755AAB
:1045F60002755B00AE52AF53E53C75F00FA4FDACFF
:10460600F0EDD39FEC9E4021E53C8E048F05FF1212
:104616006FC7ED75F010A4FFAEF0E55F75F011847D
:10462600FD7C00ED2FF53D800EE55F75F01184FFF2
:104636007E00EF24F0F53D853D37E55F75F011848A
:10464600AFF07E008F3A12429785373EAE52AF5397
:104656009000F9E075F00FA4FDACF0EDD39FEC9E51
:104666004028755A02755B10853D37124297853E84
:1046760038853739AE52AF53E53C8E048F05FF12AD
:104686006FF28D3A853C3B12431185372975280018
:10469600752B64752A00229000F9E0F53C753F11F0
:1046A600755A02755B00AE52AF53E53C75F00FA428
:1046B600FDACF0EDD39FEC9E4021E53C8E048F05CA
:1046C600FF126FC7ED75F010A4FFAEF0E56175F04F
:1046D6001184FD7C00ED2FF53D800EE56175F0112E
:1046E60084FF7E00EF24F0F53D853D37E56175F0EA
:1046F6001184AFF07E008F3A12429785373EAE5254
:10470600AF539000F9E075F00FA4FDACF0EDD39F28
:10471600EC9E4028755A02755B10853D371242970C
:10472600853E38853739AE52AF53E53C8E048F054A
:10473600FF126FF28D3A853C3B124311853729757E
:104746002800E56B6017E56BC394FE50109000EDF2
:10475600E0B402099000DBE0D3940B50028017AE60
:1047660028AF29E56B126FD774E78E048F05FF1209
:104776006FC78C288D299000C3E0B40453E55F759C
:10478600F00484FF7E008F37E55F75F00484ADF09A
:104796007C008D3A753F04755A01755B00E537C399
:1047A600943F500512429780069001C7E0F537AE58
:1047B60028AF29E537126FD774648E048F05FF1270
:1047C6006FC7AE28AF29EF2DFDEE3CFC8C288D2956
:1047D600752B64752A002290008EE0B40146E567C9
:1047E60075F00A84FF7E008F37E56775F00A84ADA1
:1047F600F07C008D3A753F0A755A05755B00E53702
:10480600C3941150051242978006900599E0F5373A
:10481600AE2AAF2BE5372FFF50010E746412701AC3
:104826008E2A8F2B90008FE0B40146E56875F00A5A
:1048360084FF7E008F37E56875F00A84ADF07C0052
:104846008D3A753F0A755A05755B6CE537C3941149
:1048560050051242978006900605E0F537AE2AAF5E
:104866002BE5372FFF50010E746412701A8E2A8FB3
:104876002B90009EE0B40249E56AC3944175F005A9
:1048860084FF7E008F37E56A75F00584ADF07C0005
:104896008D3A753F05755A06755B00E537C3941367
:1048A6005005124297800690069BE0F537AE2AAF78
:1048B6002BE5372FFF50010E746412701A8E2A8F63
:1048C6002B9000E0E0B40202800302497CE55F75AC
:1048D600F01584FF7E008F37E55F75F01584ADF027
:1048E6007C008D3A753F15755A03755BF4E537C341
:1048F600940B50051242978006900487E0F537E541
:104906003775F0FFA4FFAEF09000E1E08E048F054E
:10491600FF126FC7ED900072F0E56675F078A4FFA0
:10492600AEF074FF8E048F05FF126FC78C5A8D5B35
:1049360074028C068D071200398F37AC5AAD5B7442
:1049460004FF126FF28D3A753F04755A06755B289F
:10495600E537C3941D500512429780069006CDE0B8
:10496600F537AE2AAF2BE5372FFF50010E746412D0
:10497600701A8E2A8F2B90008DE0B4025DE561756A
:10498600F064A4FFAEF074081200398E5C8F5D747B
:10499600058E048F05FF126FC78D37AE5CAF5D7451
:1049A600058E048F05FF126FF28D3A753F05755A15
:1049B60005755BDEE537C3941350051242978006F2
:1049C600900679E0F537AE2AAF2BE5372FFF500179
:1049D6000E746412701A8E2A8F2B9000CFE0703CF2
:1049E60090005CE075F00584FF7E008F3790005CD8
:1049F600E075F00584ADF07C008D3A753F05755A7B
:104A060005755BC0E537C3941D50051242978006B5
:104A1600900665E0F537E53790007AF0229000962B
:104A2600E0B401179008B5E0252BFFAE2A50010E21
:104A36009000EAE012701A8E2A8F2B90010EE0B4D5
:104A4600011490010FE0A852B8000495535007E5F1
:104A56005FC39560400280139000B8E0252BFFAE3F
:104A66002A50010E8E2A8F2B024E52900096E0B4E9
:104A76000306A22AB3B3400280509008BEE070102D
:104A86009008B8E0C39405A852B8000695534002B2
:104A960080109000B8E0252BFFAE2A50010E8E2A1A
:104AA6008F2B9008BEE0600D9008B8E0A852B800C1
:104AB600069553400280109000B8E0252BFFAE2AE1
:104AC60050010E8E2A8F2B024E52900090E0B402B7
:104AD600028003024E52900093E0602FE567D39464
:104AE600464028900017E0FEA3E0FF9000CEE07558
:104AF600F003A4FDACF0EFD39DEE9C400E9000F2C7
:104B0600E0A852B80005D395535003024E529000C8
:104B1600C3E0B403028003024CB685615B755A009C
:104B260090009AE0A852B800049553500E90009B4E
:104B3600E0A85AB80005D3955B5003024CB3E56173
:104B460075F002A4FFAEF074158E048F05FF126F88
:104B5600C78C068D07900618120048FEE0FFEE90FF
:104B66000092E0FEEF8E0088F0A4FFAEF074648E33
:104B7600048F05FF126FC78C5A8D5B90005CE07541
:104B8600F018A4FFAEF09000D9E08E048F05FF1256
:104B96006FC78C068D07900630120048AE5AAF5B81
:104BA600E0126FD774648E048F05FF126FC78C5A9C
:104BB6008D5BE565A85AB80077D3955B4072E565CD
:104BC600C3955BFFE4955AFE8E5A8F5B7428BE0030
:104BD600039F500C755B28755A00740D90005DF0AC
:104BE600AE5AAF5B900093E0126FD774288E048F95
:104BF60005FF126FC78C5A8D5BAE28AF29740A8EDB
:104C0600048F05FF126FC78D068C07AC5AAD5BCFBC
:104C1600CECF120003740A8E048F05FF126FC78C65
:104C26005A8D5BAE28AF291270228E288F29807D7F
:104C3600E565A85AB80004955B5072AE5AAF5BE5BD
:104C46006512701A8E5A8F5B7428BE00039F500C33
:104C5600755B28755A00740D90005DF0AE5AAF5B17
:104C6600900093E0126FD774288E048F05FF126FA1
:104C7600C78C5A8D5BAE28AF29740A8E048F05FF48
:104C8600126FC78D068C07AC5AAD5BCFCECF120024
:104C960003740A8E048F05FF126FC78C5A8D5BAEA4
:104CA60028AF29EF2DFDEE3CFC8C288D29024E52B3
:104CB6009000DBE0855FF0A4FFAEF07405126FD7BD
:104CC60074071200398E5A8F5B90009AE0A852B88A
:104CD60000049553501290009BE075F002A4FDACC1
:104CE600F0EFC39DEE9C4003024E52E55F75F00B5C
:104CF60084FF7E00900618120048FEE0FFEE90004A
:104D060092E0FEEF8E0088F0A4FFAEF074648E048D
:104D16008F05FF126FC78C5A8D5B90005CE075F0B3
:104D260018A4FFAEF09000D9E08E048F05FF126F35
:104D3600C78C068D07900630120048AE5AAF5BE06E
:104D4600126FD774648E048F05FF126FC78C5A8D4D
:104D56005BE565A85AB80077D3955B4072E565C3F5
:104D6600955BFFE4955AFE8E5A8F5B7428BE00034E
:104D76009F500C755B28755A00740D90005DF0AE5F
:104D86005AAF5B900093E0126FD774288E048F059C
:104D9600FF126FC78C5A8D5BAE28AF29740A8E043A
:104DA6008F05FF126FC78D068C07AC5AAD5BCFCE51
:104DB600CF120003740A8E048F05FF126FC78C5A38
:104DC6008D5BAE28AF291270228E288F29807DE553
:104DD60065A85AB80004955B5072AE5AAF5BE5659C
:104DE60012701A8E5A8F5B7428BE00039F500C7582
:104DF6005B28755A00740D90005DF0AE5AAF5B905B
:104E06000093E0126FD774288E048F05FF126FC7C8
:104E16008C5A8D5BAE28AF29740A8E048F05FF125B
:104E26006FC78D068C07AC5AAD5BCFCECF12000391
:104E3600740A8E048F05FF126FC78C5A8D5BAE28DD
:104E4600AF29EF2DFDEE3CFC8C288D29229000EE3B
:104E5600E0B4026AE55F75F00884FF7E008F37E5EF
:104E66005F75F00884ADF07C008D3A753F08755A81
:104E760001755BE0E537C3943F5005124297800603
:104E8600900287E0F53785372D752C00AE2CAF2DB7
:104E9600AC2AAD2B12000374648E048F05FF126FCB
:104EA600C78C2C8D2D90008BE08C068D07126FD74A
:104EB60074648E048F05FF126FC78C2C8D2DAE285F
:104EC600AF29AC2AAD2B12000374648E048F05FF44
:104ED600126FC78C288D2990008BE08C068D0712E7
:104EE6006FD774648E048F05FF126FC78C288D29C7
:104EF600A203401DAE52AF537405BE00039F50027D
:104F0600D203E561D394CC4008D201741190005DC0
:104F1600F09000EDE0B402089000DBE0640B600264
:104F26008035AE28AF29E56B126FD774E78E048FF4
:104F360005FF126FC78C288D299000EEE0B402178A
:104F4600AE2CAF2DE56B126FD774E78E048F05FF7D
:104F5600126FC78C2C8D2D9000ADE05402601B9013
:104F660000A4E0A852B80012D39553400DA203B393
:104F7600B35007E561C3949A40028028AE34AF353A
:104F86009000A2E075F002A4FDACF0EF2DFDEE3C22
:104F9600FC74022DFD50010CE561BC0007D39D4059
:104FA60003754301856135753400E543700302508E
:104FB60096900100E0C3954350030250889001107B
:104FC600E0C394025076E56775F00A84FF7E009090
:104FD6000588120048E0F55B755A00AE5AAF5B9043
:104FE60000A3E0126FD774648E048F05FF126FC79B
:104FF6008C5C8D5D900100E004C395438C068D07A3
:10500600126FD7900100E08E048F05FF126FC78CD8
:105016005C8D5DAE28AF29EF2DFDEE3CFC8C288D16
:10502600299000EEE0B40212AE2CAF2DAA5CAB5D67
:10503600EF2BFBEE3AFA8A2C8B2D8046900100E08E
:1050460004C39543854BF0A4FFAEF0900100E08EBB
:10505600048F05FF126FC78C5C8D5DAE28AF29EFFC
:105066002DFDEE3CFC8C288D299000EEE0B402125A
:10507600AE2CAF2DAA5CAB5DEF2BFBEE3AFA8A2C79
:105086008B2D0543900100E0C39543500375430003
:105096009000ADE05401601B9000A1E0A852B8005A
:1050A60012D39553400DA203B3B35007E55FC394E3
:1050B600CC4002802590009FE075F003A4FFAEF07F
:1050C600E5402FFF50010E74032FFF50010EE55FE0
:1050D600BE0007D39F4003754401855F40E54470D9
:1050E600030251C9900101E0C3954450030251BB2C
:1050F600900110E0C394025076E56775F00A84FFCC
:105106007E00900588120048E0F55B755A00AE5A9D
:10511600AF5B9000A0E0126FD774648E048F05FF1A
:10512600126FC78C5C8D5D900101E004C395448CC1
:10513600068D07126FD7900101E08E048F05FF12CE
:105146006FC78C5C8D5DAE28AF29EF2DFDEE3CFC64
:105156008C288D299000EEE0B40212AE2CAF2DAA59
:105166005CAB5DEF2BFBEE3AFA8A2C8B2D804690DA
:105176000101E004C39544854CF0A4FFAEF0900114
:1051860001E08E048F05FF126FC78C5C8D5DAE2823
:10519600AF29EF2DFDEE3CFC8C288D299000EEE02A
:1051A600B40212AE2CAF2DAA5CAB5DEF2BFBEE3A30
:1051B600FA8A2C8B2D0544900101E0C395445003D7
:1051C600754400900103E02529FFAE2850010E8E9C
:1051D600288F299000B2E0A828B800049529500924
:1051E6009000B2E0F5297528009000EEE0B4020DBB
:1051F6009000B2E0A82CB80006952D4002800990D8
:1052060000B2E0F52D752C00229000EEE0B401020C
:10521600800302531AA203B350030253189000B935
:10522600E0B40168AE28AF29AC52AD531200037446
:105236003C8E048F05FF126FC79000C9E0BC0010BA
:105246009D400D9000CBE0A828B800049529500297
:10525600D202AE28AF29AC52AD53120003743C8E75
:10526600048F05FF126FC79000C9E0C3940ABC0003
:1052760015D39D40119000CBE0C39405A828B80033
:1052860005D3952950028002C2028068AE28AF2954
:10529600AC52AD5312000374788E048F05FF126F63
:1052A600C79000C9E0BC00109D400D9000CBE0A85F
:1052B60028B8000495295004D2028038AE28AF29B8
:1052C600AC52AD5312000374788E048F05FF126F33
:1052D600C79000C9E0C3940ABC0015D39D40119045
:1052E60000CBE0C39405A828B80005D39529500241
:1052F6008002C202A202B34019AE28AF299000CAAA
:10530600E0126FD774648E048F05FF126FC78C2866
:105316008D298002C202A200B34006A201B3B35097
:105326000990001FE4F0A3F08024AE28AF29740092
:10533600D39F74019E400C90001FE528F0A3E52939
:10534600F0800B74FF90001FF8E4F0E8A3F09000E3
:10535600B9E0B4011AAE28AF297402126FD78E28AD
:105366008F29AE2CAF2D7402126FD78E2C8F2D90F5
:1053760000D0E0C394034009900084E0C394025037
:1053860035AE28AF29745E126FD7740A8E048F0566
:10539600FF126FC78C288D299000EEE0B40217AE7D
:1053A6002CAF2D745E126FD7740A8E048F05FF1210
:1053B6006FC78C2C8D2DAE28AF297402BE000AD380
:1053C6009F4006752902752800AE2CAF2D7402BECB
:1053D600000AD39F4006752D02752C0090001DE52E
:1053E60028F0A3E529F02290005CE0900388127073
:1053F60008E0F54175426490005CE0FE9000C4E070
:10540600D39E4037E55F75F00884FF7E008F37E551
:105416005F75F00884ADF07C008D3A753F08755ACB
:1054260003755B96E537C3941F50051242978006B5
:1054360090043DE0F5378537428035E55F75F00825
:1054460084FF7E008F37E55F75F00884ADF07C0041
:105456008D3A753F08755A03755BB6E537C3941FD9
:105466005005124297800690045DE0F53785374275
:10547600229000FAE0F53C753F11755A04755B0001
:10548600AE52AF53E53C75F00FA4FDACF0EDD39FE3
:10549600EC9E4021E53C8E048F05FF126FC7ED752B
:1054A600F010A4FFAEF0E55F75F01184FD7C00ED11
:1054B6002FF53D800EE55F75F01184FF7E00EF2429
:1054C600F0F53D853D37E55F75F01184AFF07E0060
:1054D6008F3A12429785373EAE52AF539000FAE0AC
:1054E60075F00FA4FDACF0EDD39FEC9E4028755AE5
:1054F60004755B10853D37124297853E38853739EE
:10550600AE52AF53E53C8E048F05FF126FF28D3A13
:10551600853C3B124311853741754264229000FA5F
:10552600E0F53C753F11755A04755B00AE52AF53FA
:10553600E53C75F00FA4FDACF0EDD39FEC9E402149
:10554600E53C8E048F05FF126FC7ED75F010A4FFC2
:10555600AEF0E56175F01184FD7C00ED2FF53D8020
:105566000EE56175F01184FF7E00EF24F0F53D85B0
:105576003D37E56175F01184AFF07E008F3A124237
:105586009785373EAE52AF539000FAE075F00FA400
:10559600FDACF0EDD39FEC9E4028755A04755B1068
:1055A600853D37124297853E38853739AE52AF531F
:1055B600E53C8E048F05FF126FF28D3A853C3B1257
:1055C60043118537417542649000F5E0B404799043
:1055D600005CE0FE9000C4E0D39E4037E55F75F0C6
:1055E6000884FF7E008F37E55F75F00884ADF07C98
:1055F600008D3A753F08755A03755B96E537C39477
:105606001F5005124297800690043DE0F537853716
:10561600428035E55F75F00884FF7E008F37E55FD1
:1056260075F00884ADF07C008D3A753F08755A0315
:10563600755BB6E537C3941F5005124297800690F6
:10564600045DE0F5378537422290008EE0B4013BD9
:10565600E56775F00A84FF7E008F37E56775F00A07
:1056660084ADF07C008D3A753F0A755A05755B125C
:10567600E537C39411500512429780069005ABE0BA
:10568600F537E5422537C39464F54290008FE0B4C0
:10569600013BE56875F00A84FF7E008F37E5687583
:1056A600F00A84ADF07C008D3A753F0A755A05758F
:1056B6005B7EE537C394115005124297800690062B
:1056C60017E0F537E5422537C39464F542E54125F1
:1056D60042F536900096E0B402109008B4E0253604
:1056E600FE9000EAE0F4042EF5369000EDE0D39447
:1056F600014040E56BC394E7501D74E7C3956BFE0C
:105706009008B6E08E00F5F0E884FF7E008F37E55E
:10571600362537F536801CE56BC394E7FE9008B650
:10572600E08E00F5F0E884FF7E008F37E536C395FE
:1057360037F536A2034006E5412464F536E536D34F
:1057460094644009E536C39464F5368003753600E3
:105756009000C6E0C3953650069000C6E0F53622A6
:10576600D200900078E0A852B800049553503E90BD
:105776000078E0A852B800049553500375360F9090
:105786000078E004A852B800049553500375360714
:10579600900078E02402A852B8000495535002C243
:1057A60000900078E06006740990005DF0C2317EDA
:1057B600017F009000CCE0126FD79000DBE08E04F2
:1057C6008F05FF126FC7E55FBC0017D39D4013908E
:1057D60000D5E0B40204D2318002C200740A9000FF
:1057E6005DF090008EE0B401099000CDE0C39567AE
:1057F600400280159000DFE0A852B800049553508F
:1058060002C200740B90005DF090008EE0B40107B8
:10581600E567C394644002801D900125E0600D9009
:105826000125E0A852B80006955340028008C20040
:10583600740B90005DF0A200400375360090010ED7
:10584600E0B4011490010FE0A852B800049553503B
:1058560007E55FC39560400280209000B7E0D394CF
:105866001D400B9000B7E0C3941EF53680037536D5
:1058760000741590005DF0025957900096E0B4034D
:1058860006A22AB3B340030259579008B8E0C3945E
:1058960005A852B80004955350069008BEE0600271
:1058A600801D9000B7E0D3941D400B9000B7E0C375
:1058B600941EF5368003753600740C90005DF090EA
:1058C60008B8E0A852B80004955350069008BEE008
:1058D6007002801D9000B7E0D3941D400B9000B776
:1058E600E0C3941EF5368003753600740C90005D97
:1058F600F09008B8E0A852B80004955350319000D3
:10590600D5E0B40228D2319008BDE0FE9008BEE092
:10591600D39E50069008BEE0700280099008BDE450
:10592600F0C23180069008BDE004F08002C200900B
:1059360008B8E02405A852B8000495535013900007
:10594600D5E0B4020A9008BEE07002D2318002C2ED
:1059560000A230B3401D9000B7E0D3941D400B90D9
:1059660000B7E0C3941EF5368003753600741090B8
:10597600005DF085366C9000B7E0D3941D4018901A
:105986000085E02536FE90005CE075F01E84FC7F05
:1059960000EE2CF536804990005DE0640C600F90B7
:1059A600005DE06410600790005DE0B4151690009D
:1059B60085E0FE90005CE075F01E84FC7F00EE2C16
:1059C600F536801C900087E02536FE900085E02E97
:1059D600FE90005CE075F01E84FC7F00EE2CF53630
:1059E6002290005CE075F00584FF7E008F37900002
:1059F6005CE075F00584ADF07C008D3A753F057569
:105A06005A03755BD69000D9E01475F00584FF7EC5
:105A160000E537BE00039F5005124297800BE5371D
:105A260090045E127008E0F537E5379008B7F090FD
:105A360008B7E0FE9000C8E0C39E50089000C8E09A
:105A46009008B7F022E56775F00A84FF7E0090059E
:105A560088120048E0F546E546D394644010E546D2
:105A6600C3946475F00F84FF7E008F4680037546ED
:105A7600009000ABE02546F54622E56775F00A84FE
:105A8600FF7E00900588120048E0C3946950559047
:105A960000F5E0C39403502690088AE0FEA3E0FFD9
:105AA6007404120039E55F126FD7740F8E048F05E8
:105AB600FF126FC7900888ECF0A3EDF080249008E1
:105AC6008AE0FEA3E0FF7404120039E561126FD785
:105AD600740F8E048F05FF126FC7900888ECF0A331
:105AE600EDF0800F90088AE0F8A3E0900888C8F0EF
:105AF600A3C8F0A203401A90088AE0FEA3E0FF7450
:105B060003126FD77401120039900888EEF0A3EFE4
:105B1600F0900888E0FEA3E0FF90088EE0FCA3E08A
:105B2600FDEDD39FEC9E400F90088EE0F8A3E09029
:105B36000888C8F0A3C8F090009EE0B40262E56A47
:105B4600C3944175F00584FF7E008F37E56A75F0D2
:105B56000584ADF07C008D3A753F05755A06755B78
:105B660014E537C39417500512429780069006AF86
:105B7600E0F537900888E0FEA3E0FF740A8E048FF4
:105B860005FF126FC7E5378C068D07126FD7740AAB
:105B96008E048F05FF126FC7900888ECF0A3EDF016
:105BA60022E50875F004A4FFAEF09006CB1200487B
:105BB600E09068DBF8282873804C85537380479003
:105BC60000DBE0855FF0A4FFAEF074081200398FA9
:105BD600738033856173802E85677380298568732A
:105BE6008024856973801F856A73801A856B73802C
:105BF600158566738010856573800B856C738006CA
:065C0600900020E0F573A0
:1068DB00025BBE025BC0025BC5025BD9025BDE02E0
:1068EB005BE3025BE8025BED025BF2025BF7025BD0
:0768FB00FC025C01025C06D7
:105C0C00E50875F004A4FFAEF09006CC120048E550
:105C1C000875F004A4FFAEF0E0FC9006CD1200482D
:105C2C00ECFEE0FFEEC39F4003025D14E50875F047
:105C3C0004A4FFAEF09006CB120048E0B40441E59A
:105C4C000875F004A4FFAEF09006CD120048E0C336
:105C5C009573500AE508F50CD39232120EC8E5087C
:105C6C0075F004A4FFAEF09006CC120048E0D3957A
:105C7C0073400AE508F50CC39232120EC8025D128D
:105C8C00E50875F004A4FFAEF09006CC120048E0D5
:105C9C00C395735015E50875F004A4FFAEF090069B
:105CAC00CD120048E0D395735002800AE508F50C3C
:105CBC00D39232120EC8E50875F004A4FFAEF09032
:105CCC0006CC120048E0D395735015E50875F00426
:105CDC00A4FFAEF09006CD120048E0C39573500AB5
:105CEC00E508F50CC39232120EC89006D3E0B4014D
:105CFC00099000E7E0D395615002800A7402F50C1C
:105D0C00C39232120EC8806AE50875F004A4FFAE87
:105D1C00F09006CC120048E0D395734015E5087559
:105D2C00F004A4FFAEF09006CD120048E0C39573CA
:105D3C004002800AE508F50CC39232120EC8E50841
:105D4C0075F004A4FFAEF09006CC120048E0C395A9
:105D5C00734015E50875F004A4FFAEF09006CD1263
:105D6C000048E0D39573400AE508F50CD392321243
:105D7C000EC822AE2EAF2F74C9BE000CD39F4008A4
:105D8C00782E12702A025E99752F01752E00AE5274
:105D9C00AF53E546BE000DD39F40099000BDE0D344
:105DAC00954740028023754700E546C39553F5732C
:105DBC009000C0E0D395454008E5452573F5458036
:105DCC00069000C0E0F54580020547900099E0D3AD
:105DDC009561401CE55FC395604015AE52AF53E52D
:105DEC0046BE00039F50099000BEE0D39548400288
:105DFC00806E9008B9E0A852B80004955350037512
:105E0C004A009008B9E0A852B8000BD3955340064D
:105E1C00E5539008B9F0E54A7041E553C39546F552
:105E2C0073E573D3940540037573059000BFE0C30D
:105E3C0095455007E573C3954540028009E545C378
:105E4C009573F54580069000BFE0F5459000BFE0E6
:105E5C00D3954540069000BFE0F54575480080029B
:105E6C000548E54A7016900099E0C39561500DE520
:105E7C00462405A852B8000695534002800F9000A6
:105E8C00ACE0F545754A0174789008B9F022AE2E55
:105E9C00AF2F74E9D39F74039E4008782E12702A9A
:105EAC00026040752F01752E00754532A22B402AD9
:105EBC007545199000ACE075F002A4FFAEF0E54713
:105ECC00BE0006D39F4002D22B0547754A03747857
:105EDC009008B9F0754900026027AE52AF53E54601
:105EEC006F4E7003026027E546BE000DD39F40093C
:105EFC009000BDE0D395474002800F754700E54AFE
:105F0C00C394035003754519800DE546C39553F5AD
:105F1C0073E5472573F547900099E0D39561400EE2
:105F2C009008B9E0A852B80007D395534002800CF2
:105F3C0005499000ACE0B54903754A00E54AB40345
:105F4C0006A203B3B34002800A0549E549B43C03F9
:105F5C00754A02E54AB402299008B9E0A852B80083
:105F6C000ED395534009E5539008B9F0754900904C
:105F7C000099E0C39561500975490074789008B98F
:105F8C00F0E54A705A900099E0D39561401CE55FAA
:105F9C00C395604015AE52AF53E546BE00039F500B
:105FAC00099000BEE0D39548400280087548007502
:105FBC00454B8028E553C39546F573E573D394059B
:105FCC004003757305900099E0D395614008E5484E
:105FDC002573F5488006E5482406F548754900E523
:105FEC004A7016900099E0C39561500DE546240562
:105FFC00A852B80006955340028003754A01E54A41
:10600C00B4011875451905499000ACE0B549067501
:10601C004A0275490074789008B9F0A201B34003A4
:10602C00754532E54575F00AA4FFAEF0900890EE88
:10603C00F0A3EFF022E56F906902F8282873900026
:10604C0091E0700302627E9000C7E0B4010280030D
:10605C0002618990005AE0655E6009E55345526023
:10606C00030261867E017F00E5BE126FD7E5BD2F6E
:10607C00FF50010E8E5A8F5B7410126FD790007701
:10608C00E08E048F05FF126FC7900894ECF0A3ED1F
:10609C00F0E56B600FE56BC394FE50089000EDE0EB
:1060AC006402600280649000DBE0B40B1F900894E3
:1060BC00E0FEA3E0FF74E7126FD7E56B8E048F054B
:1060CC00FF126FC7900894ECF0A3EDF09000DBE0AA
:1060DC00D3940B40089000C3E064046002802B90C2
:1060EC000894E0FEA3E0FF900898E0FCA3E0FDEF2D
:1060FC00D39DEE9C400D127022900894EEF0A3EF0D
:10610C00F08007900894E4F0A3F0900091E0B402C2
:10611C0027900896E0FEA3E0FF900894E0FCA3E033
:10612C00FDEF2DFDEE3CFC74018C068D0712003941
:10613C00900894EEF0A3EFF0900894E0FEA3E0FF3B
:10614C00900896E0FCA3E0FDEDD39FEC9E4004D2BA
:10615C002F8002B22F900894E0F8A3E0900896C824
:10616C00F0A3C8F09000C3E064016006A22FB3B3A3
:10617C0040028006900895E0F55F02627CD22F7E8B
:10618C00017F00E5BE126FD7E5BD2FFF50010E8ECB
:10619C005A8F5B7410126FD7900077E08E048F05C6
:1061AC00FF126FC7900894ECF0A3EDF0E56B600F55
:1061BC00E56BC394FE50089000EDE0640260028031
:1061CC00649000DBE0B40B1F900894E0FEA3E0FFAA
:1061DC0074E7126FD7E56B8E048F05FF126FC790B3
:1061EC000894ECF0A3EDF09000DBE0D3940B4008A6
:1061FC009000C3E064046002802B900894E0FEA33E
:10620C00E0FF900898E0FCA3E0FDEFD39DEE9C40EE
:10621C000D127022900894EEF0A3EFF08007900816
:10622C0094E4F0A3F0900091E0B40227900896E07B
:10623C00FEA3E0FF900894E0FCA3E0FDEF2DFDEE43
:10624C003CFC74018C068D07120039900894EEF01A
:10625C00A3EFF0900894E0F8A3E0900896C8F0A3A0
:10626C00C8F09000C3E064016006900895E0F55F0B
:10627C008003755F0090008DE07006756F01026001
:10628C004175BB180268B590008DE0700302640480
:10629C007E017F00E5BE126FD7E5BD2FFF50010ECA
:1062AC008E5A8F5B9000D3E0B4010F7E0F7FFFAC52
:1062BC005AAD5B1270228E5A8F5B9000F8E0B402DC
:1062CC0045AE5AAF5B900029E0FCA3E0FDEDD39FF7
:1062DC00EC9E400A900029E55AF0A3E55BF0AE5A1B
:1062EC00AF5B90002BE0FCA3E0FDEFD39DEE9C4058
:1062FC000A90002BE55AF0A3E55BF0AE5AAF5B7445
:10630C00041200398F619000F8E0704CAE5AAF5B0C
:10631C00900029E0FCA3E0FDEFD39DEE9C40091218
:10632C0070228E5A8F5B8006755B00755A00AE5AD0
:10633C00AF5B7410126FD7900074E08E048F05FF62
:10634C00126FC78C5A8D5B74FFBC0009D39D40053E
:10635C00855B6180037561FE9000C3E0B40102802F
:10636C0003026402A203B3B3500E900097E0A8524C
:10637C00B80005D39553500280719000D4E085612C
:10638C00F0A4FFAEF074648E048F05FF126FC78CFF
:10639C005A8D5BE56B6016E56BC394FE500F900055
:1063AC00EDE0B402089000DBE0640B60028017AEF5
:1063BC005AAF5B74E7126FD7E56B8E048F05FF1233
:1063CC006FC78C5A8D5BAE5AAF5B900894E0FCA300
:1063DC00E0FDEDD39FEC9E4005855B5F800BA22F0B
:1063EC00B34006900895E0F55F800BA22FB34006F2
:1063FC00900895E0F55F8003756100900090E07067
:10640C0006756F0202604175BB190268B590009069
:10641C00E070030264B9E55ED3955140030264B7A2
:10642C00900027E0FEA3E0FFE56512701A900027AC
:10643C00EEF0A3EFF07E017F00E5BE126FD7E5BD55
:10644C002FFF50010E8E5A8F5B9000FDE07013747D
:10645C000A126FD774518E048F05FF126FC78D65AA
:10646C008019AE5AAF5B740A126FD78F048E057EFB
:10647C00017F95CDCCCD126EC58F65E565D3946447
:10648C004003756564900027E0FEA3E0FFE5652FEF
:10649C00FF50010E900027EEF0A3EFF0900094E077
:1064AC00048E048F05FF126FC78D658003756532EE
:1064BC009000E0E07006756F0302604175BB13023B
:1064CC0068B59000E0E0604A7E017F00E5BE126F87
:1064DC00D7E5BD2FFF50010E8E5A8F5B740412004E
:1064EC00398F669000E2E08566F0A4FDACF0746430
:1064FC00FF126FC78D669000E1E08566F0A4FFAED9
:10650C00F074FF8E048F05FF126FC7ED900073F0CF
:10651C00800375660090008EE07006756F04026053
:10652C004175BB170268B590008EE0B40102800380
:10653C000265C77E017F00E5BE126FD7E5BD2FFF58
:10654C0050010E8E5A8F5B9008BAE060199008BA11
:10655C00E0149069D212008CE493FC740193FDED6D
:10656C00C39FEC9E400280069008BAE014F090089D
:10657C00BAE0C394B3501DAE5AAF5B9008BAE004B6
:10658C009069D212008CE493FC740193FDEFC39DCF
:10659C00EE9C400280069008BAE004F09008BAE045
:1065AC00FE9000B4E08E0088F0A4FFAEF074648E10
:1065BC00048F05FF126FC78D67800375670090000D
:1065CC008FE07006756F0502604175BB160268B5E9
:1065DC0090008FE0B4010280030266707E017F00A0
:1065EC00E5BE126FD7E5BD2FFF50010E8E5A8F5BA3
:1065FC009008BBE060199008BBE014906B3C120053
:10660C008CE493FC740193FDEDC39FEC9E400280DF
:10661C00069008BBE014F09008BBE0C394B3501D87
:10662C00AE5AAF5B9008BBE004906B3C12008CE45C
:10663C0093FC740193FDEFC39DEE9C400280069089
:10664C0008BBE004F09008BBE0FE9000BAE08E00BE
:10665C0088F0A4FFAEF074648E048F05FF126FC730
:10666C008D68800375680075BB1F0268B57E017F5D
:10667C0000E5BE126FD7E5BD2FFF50010E8E5A8F6D
:10668C005B7409126FD774E68E048F05FF126FC707
:10669C008D6A900096E07006756F0702604175BBBD
:1066AC00150268B5900096E070030268017E017FC8
:1066BC0000E5BE126FD7E5BD2FFF50010E8E5A8F2D
:1066CC005B74041200398F69900096E0B401159048
:1066DC0000EAE08569F0A4FFAEF07407120039EF10
:1066EC009008B5F0900096E0B402159000EAE085B1
:1066FC0069F0A4FFAEF07407120039EF9008B4F003
:10670C00900096E0B4030280030267E49000D7E0A7
:10671C007052E569C39419500FD22A9000B6E090DC
:10672C0008B8F09008BCE4F0E569D394644004A286
:10673C002A4002802D9008BCE004F09008BCE0FEDA
:10674C00900129E0B5060B9008B8E004F09008BC65
:10675C00E4F09008B8E064966006900129E07002BD
:10676C00C22A80639000B6E070349000EAE085693C
:10677C00F0A4FFAEF074FF8E048F05FF126FC7ED0F
:10678C009008B8F0AE52AF53741EBE0006D39F40B3
:10679C0002D22AE561D394E54002C22A8029E56938
:1067AC00C3940A500DAE52AF53741EBE0004D39F57
:1067BC0050028002D22AE561D394E54002C22A90AD
:1067CC0000B6E09008B8F09008B8E0C39405500605
:1067DC0074059008B8F0C230900096E0B40414E54B
:1067EC0069C394195002D230E569D394324002C285
:1067FC0030C22A80037569009000EDE07006756F59
:10680C000802604175BB140268B59000EDE070039E
:10681C000268A47E017F00E5BE126FD7E5BD2FFF95
:10682C0050010E8E5A8F5B900112E07025EFD394BD
:10683C0021EE940E4005756BFF8015AE5AAF5B745C
:10684C0010126FD774E38E048F05FF126FC78D6B18
:10685C008027AE5AAF5BEFD39449EE940640057592
:10686C006BFF8015AE5AAF5B7410126FD774658EC8
:10687C00048F05FF126FC78D6BE56B75F00BA4FFD2
:10688C00AEF09000DBE08E048F05FF126FC790080E
:10689C0098ECF0A3EDF08003756B00900091E06034
:0968AC000575BB1A800375BB18C9
:1069020002604A0262930264190264CE0265330293
:0B69120065DC0266790266B0026816C0
:0568B500056FD2EC228A
:097008002582F582500205832265
:0F008C0025E050020583258250020583F582226C
:106FA600EF2F500205832582F582E5833E2EF58379
:016FB60022B8
:10701A00CFC39FFF50011E22C3EF9DFFEE9CFE22AD
:08702A000806B6000218062258
:0D6FE500A3E004F07006126FFEE004F0223D
:0E003900048007C3CE13CECF13CFD5E0F6223E
:106EC500BC000FBE0008ED8FF084FFADF022E4FE9C
:106ED500FF22BE000DEF60FE54F0606F20E7030255
:106EE5006F7BEAC0E0EBC0E078017A0075F001EE57
:106EF50020E710EF25E0FFEE33FE0AC5F023C5F0CD
:106F050030E7F0EA5407F9096A7A007B0060010866
:106F1500C3EC9E40167004ED9F4010ED9FFDEC9E66
:106F2500FCE5F0CA4ACA03F5F08005E5F003F5F083
:106F3500C3EE13FEEF13FFD9D77908CACBCAD8D051
:106F4500EAFEEBFFD0E0FBD0E0FA22EC8FF084FC08
:106F5500ED54F045F0C48FF084FEEDC454F045F0D7
:106F6500C48FF084FDEEC4FE54F02DFFEE540F3CAB
:106F7500FEADF07C0022790078008FF0EC7E0820D1
:106F8500E70DC3CD33CD33C933C9C833C8DEF0846B
:106F950049F9E5F08FF0BE00E6FD7C00E9FFE8FE6B
:016FA50022C9
:0E6FD700F88FF0A4FFE5F0CE88F0A42EFE2285
:10000300EF8DF0A4F9A8F0EF8CF0A428F8EE8DF0B2
:06001300A428FEE9FF2213
:106FB700600D782B026FC1007830D8FED5E0F8223B
:106FC700EEC0E07E00126EC5EFFDEEFCD0E0FE22C3
:0C6FF200EEC0E07E00126EC5D0E0FE2272
:03001B0002001EC2
:0300530002005652
:03009B00020071EF
:030000000270117A
:0970110075817575D00002117340
:0B004800E5822FF582E5833EF5832260
:0A6FFE000582D58202158315822258
:10001E00C0E0C0F0C083C082C0D075D0001210798D
:0B002E00D0D0D082D083D0F0D0E032E0
:10005600C0E0C0F0C083C082C0D075D00012107C52
:10006600D0D0D082D083D0F0D0E032C0E0C0F0C093
:1000760083C082C0D075D000121126D0D0D082D0D5
:0600860083D0F0D0E0324F
:00000001FF
